:100000000C9489070C94AF070C94AF070C94AF07BE
:100010000C94AF070C94AF070C94AF070C94AF0788
:100020000C94AF070C94AF070C9418090C94340986
:100030000C94AF070C94AF070C94AF070C94AF0768
:100040000C94AF070C94AF070C94AF070C94AF0758
:100050000C94AF070C94AF070C94AF070C94AF0748
:100060000C94AF070C94AF070C94AF070C94AF0738
:100070000C94AF070C94AF070C94AF070C94AF0728
:100080000C94AF070C94AF070C94AF070C94AF0718
:100090000C94AF070C94AF070C94AF070C94BF0AF5
:1000A0000C94FC0A0C94390B0C94760B0C94AF074F
:1000B0000C94AF070C94AF070C94AF070C94AF07E8
:1000C0000C94AF070C94AF070C94AF070C94AF07D8
:1000D0000C94AF070C94AF070C94AF070C94AF07C8
:1000E0000C94AF070C94AF070C94AF070C94AF07B8
:1000F0000C94AF070C94AF070C94AF070C94AF07A8
:100100000C94AF070C94AF070C94AF070C94AF0797
:100110000C94AF070C94AF070C94AF070C94CB0969
:100120000C94080A0C94450A0C94820A0C94AF07AC
:100130000C94AF070C94AF070C94AF070C94AF0767
:100140000C94AF070C94AF070C94AF070C94AF0757
:100150000C94AF070C94AF070C94AF070C94AF0747
:100160000C94AF070C94AF070C94AF070C94AF0737
:100170000C94AF070C94AF070C94AF070C94AF0727
:100180000C94AF070C94AF070C94AF070C94AF0717
:100190000C94AF070C94AF070C94AF070C94AF0707
:1001A0000C94AF070C94AF070C94AF070C94AF07F7
:1001B0000C94AF070C94AF070C94AF070C94AF07E7
:1001C0000C94AF070C94AF070C94AF070C94AF07D7
:1001D0000C94AF070C94AF070C94AF070C94AF07C7
:1001E0000C94AF070C94AF070C94AF070C94AF07B7
:1001F0000C94AF07AB1FA81FA51FA21F9F1F9C1F1A
:10020000991F961F931F901F8D1F8A1F871F841F82
:10021000811F7E1F7B1F781F751F721F6C1F6F1F32
:100220003C696E70757420747970653D22737562D7
:100230006D697422207374796C653D226865696705
:1002400068743A203530707822206E616D653D22E9
:10025000746F67676C65222076616C75653D224C12
:10026000454434222F3E266E627370266E62737090
:100270003C696E70757420747970653D2273756287
:100280006D697422207374796C653D2268656967B5
:1002900068743A203530707822206E616D653D2299
:1002A000746F67676C65222076616C75653D224CC2
:1002B000454435222F3E266E627370266E6273703F
:1002C0003C696E70757420747970653D2273756237
:1002D0006D697422207374796C653D226865696765
:1002E00068743A203530707822206E616D653D2249
:1002F000746F67676C65222076616C75653D224C72
:10030000454436222F3E266E627370266E627370ED
:100310003C696E70757420747970653D22737562E6
:100320006D697422207374796C653D226865696714
:1003300068743A203530707822206E616D653D22F8
:10034000746F67676C65222076616C75653D224C21
:10035000454437222F3E266E627370266E6273709C
:100360003C2F6669656C647365743E3C2F666F72E2
:100370006D3E3C2F74643E3C74643E266E62737026
:100380003B3C2F74643E3C2F74723E3C2F74616280
:100390006C653E3C2F74643E3C74642077696474E1
:1003A000683D323025253E3C2F74643E3C2F7472EC
:1003B0003E3C2F7461626C653E3C2F626F64793EF7
:1003C0003C2F68746D6C3E003C74723E3C74643E1D
:1003D0003C666F726D206D6574686F643D22676561
:1003E00074223E3C696E70757420747970653D228C
:1003F0007375626D697422207374796C653D22682F
:1004000065696768743A2035307078222076616CAF
:1004100075653D2252656672657368222F3E3C2FDA
:10042000666F726D3E3C2F74643E3C2F74723E3C8E
:100430002F7461626C653E3C62723E3C666F726D09
:100440002069643D22666F726D226E616D653D228A
:10045000666F726D22206D6574686F643D226765FA
:10046000742220616374696F6E3D22696E646578E1
:100470002E68746D6C223E3C6669656C64736574AD
:10048000207374796C653D2277696474683A20330F
:1004900030303B223E3C6C6567656E643E4C4544A3
:1004A00020636F6E74726F6C3C2F6C6567656E6451
:1004B0003E3C696E70757420747970653D22737569
:1004C000626D697422207374796C653D2268656978
:1004D0006768743A203530707822206E616D653D12
:1004E00022746F67676C65222076616C75653D22AA
:1004F0004C454430222F3E266E627370266E627326
:10050000703C696E70757420747970653D227375E6
:10051000626D697422207374796C653D2268656927
:100520006768743A203530707822206E616D653DC1
:1005300022746F67676C65222076616C75653D2259
:100540004C454431222F3E266E627370266E6273D4
:10055000703C696E70757420747970653D22737596
:10056000626D697422207374796C653D22686569D7
:100570006768743A203530707822206E616D653D71
:1005800022746F67676C65222076616C75653D2209
:100590004C454432222F3E266E627370266E627383
:1005A000703C696E70757420747970653D22737546
:1005B000626D697422207374796C653D2268656987
:1005C0006768743A203530707822206E616D653D21
:1005D00022746F67676C65222076616C75653D22B9
:1005E0004C454433222F3E266E627370266E627332
:1005F000703C703E003C2F74643E3C74643E3C6230
:100600003E3C2F623E3C2F74643E3C2F74723E0091
:100610003C74723E3C74643E54656D7065726174E6
:100620007572653A20003C2F74643E3C74643E3C15
:10063000623E3C2F623E3C2F74643E3C2F74723EFF
:10064000003C74723E3C74643E4D414320416464FE
:10065000726573733A20003C2F74643E3C74643EB0
:100660003C623E3C2F623E3C2F74643E3C2F7472D1
:100670003E003C74723E3C74643E495020416464C8
:10068000726573733A2000485454502F312E302035
:10069000323030204F4B0A5365727665723A2077BC
:1006A0006C705F68747470640A436F6E74656E7406
:1006B0002D747970653A20746578742F68746D6C48
:1006C0000A0A3C21444F43545950452048544D4C4C
:1006D000205055424C494320222D2F2F5733432F72
:1006E0002F4454442048544D4C20342E3031204661
:1006F00072616D657365742F2F454E2220226874D8
:1007000074703A2F2F7777772E77332E6F72672F8B
:1007100054522F68746D6C342F6672616D65736509
:10072000742E647464223E3C68746D6C3E3C686553
:1007300061643E3C7469746C653E6F574C2070690F
:10074000636F204854545020576562207365727659
:1007500065723C2F7469746C653E3C2F68656164FA
:100760003E3C626F6479207374796C653D666F6E90
:10077000742D66616D696C793A617269616C3E3C99
:100780007461626C653E3C74723E3C7464207769AF
:100790006474683D3130303E3C2F74643E3C746478
:1007A0003E3C7461626C653E3C74722076616C699B
:1007B000676E3D22746F70223E3C746420776974CA
:1007C000683E3C696D67207372633D226C6F676F92
:1007D0002E6769662220626F726465723D22302244
:1007E00020616C743D226C6F676F227469746C6554
:1007F0003D226C6F676F223E3C2F74643E3C2F7429
:10080000723E3C74723E3C74642077696474683D47
:1008100022353030223E3C68323E576562205365B7
:10082000727665722072756E6E696E67206F6E20CB
:100830006F574C207069636F3C2F68323E3C703EAE
:100840005468652077656220706167652069732050
:1008500073657276656420627920776C705F687466
:10086000747064207573696E6720746865205350D6
:100870004238303020574C414E206D6F64756C65A6
:1008800020616E6420746865206F574C2D70696319
:100890006F26636F70793B20536F66747761726562
:1008A000204150493B206120756E69717565205764
:1008B000692D466920736F6C7574696F6E2066725E
:1008C0006F6D203C623E48264420576972656C6516
:1008D00073732041423C2F623E2E3C2F703E3C6899
:1008E000723E3C7461626C653E004749463839612E
:1008F00045017B00A10000FFFFFF0066990000009A
:10090000FFFFFF21FE114372656174656420776902
:1009100074682047494D50002C0000000045017BC1
:10092000000002FE848FA9CBED0FA39CB4DA8BB339
:10093000DEBCFB0F86E24896E689A6EACAB6EE0B55
:10094000C7F24CD7F68DE7FACEF7FE0F0C0A87C434
:10095000A2F1884C2A97CCA6F3098D4AA7D4AAF510
:100960008A6505B6DCAEF70B0E8BC76471F60C2DED
:10097000ABD7EC36190D3FBAE7F4FA3B8EFFD9F747
:100980007C7BFE9FD32738C80668384398A8187622
:10099000D8D8B2081919E048792279A958A929822A
:1009A000D929B809DAE139CA176A8A419A4A77CA55
:1009B0003AA1FAEAD62AEB005BAB368BAB60BB6B95
:1009C00096EB0BC01BECF5EB2B6CBC458C7B6C9C4D
:1009D0003CBB2CDC2CFB1C1CDD3ACD5BCD7ABD9BDB
:1009E0007DBA6DDB6DFA5D1B1E3A0E5B0E7AFE9AC8
:1009F000BEB9AEDAAEF99E1A5F394F5A4F793F9AB7
:100A0000EFB8EFD9AFD1BF4E010F0DC454D0D0C154
:100A10004B09012D94D4F0CFC34811F34C845411E9
:100A2000CF1DFE5D601A8CF158A6421B04024A9A43
:100A300014B0E0E4C9942A511E68290366B88D09F0
:100A40001831B0F980A6AB5B2465F6F4F9122800E2
:100A5000A12D8836D3790027C761123E5EE0195474
:100A6000A5829625A70A35BA022B31A40694D6642E
:100A7000DAB4D7539D5413503569F6AAD4185A7F67
:100A80007105D6F126D8B07151398DBAF26759BDCA
:100A900068F9BA84D1B6D8DDAF5F4072913B69691D
:100AA000E10C64D59E4DBB7647E05C6FBD22987B20
:100AB000199962CC490FD3128BB7AF81B355FDFAA8
:100AC00098AC6C70E6C50B58AFDECCB96B6CD996A0
:100AD000F70E255DFA76E4D07F47FBCCCB12788306
:100AE000C9A879E77EF0B847E5BAB05B2726CC7C89
:100AF0007517C4D17503C79DDB366FC82B8962EFAC
:100B0000CDFD7878ED56B10FFFCEE3ADC8D9CE411B
:100B10004BF7DCDEB5EFC8E8E70BB72FBE2CD0EF04
:100B2000F7FEF183F78F5B70FC95376020AAD9C57B
:100B3000DE7BD5D1361D75B1FD661E8004E65720DB
:100B400080018E2760851692365E8438A847C18260
:100B5000D0B9D7197B245A87964C2AEEB69D5FDA16
:100B6000F1C7228AFFC1789F63C2D9289A0D20EE6F
:100B7000045F4E21C5D7E3880D7628A37F32FE5748
:100B8000A48B10C6481E8EE21D69DA04C5DDB023B1
:100B90005DCF41009F8822C2B5A07E6BC1449E916B
:100BA0004A228995931866D85B98E7C5E843951162
:100BB0000489E0950ACA39A7661DDAA6618BC621A9
:100BC00079248C51EE59619E63F6F7E1810C0EB9E0
:100BD0001407B36D79629F377A78E69E0CD0B81F00
:100BE0008B94EE46239A1CEAB09C7C9921C6239DE7
:100BF00087DA091B9C1BE658DF84E0A9792AA44EFA
:100C0000663A289BB016DAA8659D01F926A2733AC8
:100C1000385BAA8EE6F8A784935E8AAAA5C43EF93B
:100C2000FE2BA1C9024B43A7268AEAA990BC1A262B
:100C300022A4AD0E5BA356AC3A60A6079B22F76DCB
:100C40000DCEEAFA2990A46E469D8FB69EAA2A9BE5
:100C5000491AB7A6B2DC1AEB6E0653BEABA3A15C71
:100C60003E6B188F1BE8FB6BBBCCEA29ACA6AB76BE
:100C70002BA98B146CABAA81B5322A2A63115BB9FC
:100C8000E58583C64B61BDCB7AC724B109EB991CBE
:100C9000C1E2EABB2E971E984A71C521DFC927BE63
:100CA00050622C28C794B21CAEC7B4AE5B32B916E2
:100CB000E89CAB7AE18E093391F3FAD9B0C02BB737
:100CC000FAAAC554920C31CAEDBD37D68FD8BAFBFB
:100CD00073B02F83AB74A4460F0C28D5828EFC70A2
:100CE000B4A34EBC6F8309960AF0D59A0E0D2CC39F
:100CF00045B38DACD0111C0D73CBF95E9448467191
:100D0000E09D89DE68F09DB7DF67004E88E08313C1
:100D1000FE89E158209EB8E25630DE87E35740ADA9
:100D20005E8AE45550BE87E597635E87E65470DEC1
:100D3000B9E75280BE8AE851903E87E9A7A33E9268
:100D4000EA4FB0DEBAEB4DC05E88ECB3D30E95ED42
:100D50004AE09EBBEE48F02EB5EFBF039FB6F040D1
:100D6000105FBCF16D225FB2F27A30BFA5F3CB43C6
:100D70007FB6F43B505FBDF59C62EFB4F6CA714F8D
:100D8000B6F7D7832F3E11E4976F3EF6E8A74FFDE5
:100D9000FAEC23EF7E11CCC72F3FF1F41B01FCFDD1
:100DA000C3B3AE7F12A4F77F3BC601F0730719A04F
:100DB000010F88C0042A70810C6CA0031F08C108B1
:100DC0004A708214ACA0052F8841CD1500003B4825
:100DD0005454502F312E3020323030204F4B0A5394
:100DE00065727665723A20776C705F6874747064AF
:100DF0000A436F6E74656E742D747970653A20695C
:100E00006D6167652F6769660A0A00485454502F60
:100E1000312E30203430342046696C65206E6F747A
:100E200020666F756E640A5365727665723A207734
:100E30006C705F68747470640A436F6E74656E746E
:100E40002D747970653A20746578742F68746D6CB0
:100E50000A0A3C68746D6C3E3C686561643E3C7493
:100E600069746C653E6F574C207069636F204854FD
:100E7000545020576562207365727665723C2F74FA
:100E800069746C653E3C2F686561643E3C626F64CA
:100E9000793E3C68323E343034202D205061676505
:100EA000206E6F7420666F756E643C2F68323E3C16
:100EB000703E536F7272792C207468652070616780
:100EC0006520796F75206172652072657175657333
:100ED00074696E6720776173206E6F7420666F751A
:100EE0006E64206F6E207468697320736572766516
:100EF000722E3C2F703E3C2F626F64793E3C2F680F
:100F0000746D6C3E006364696E6F70737578585BC6
:100F1000000011241FBECFEFDFE3DEBFCDBF00E036
:100F20000CBF18BE19BE1ABE1BBE10E3A0E0B0E293
:100F3000EEE5F0EA00E00BBF02C007900D92A03092
:100F4000B107D9F71BBE10E3A0E0B0E301C01D92CA
:100F5000AA34B107E1F70E942B430C942D500C9456
:100F600000009BB78BBFFB018091CA014093CA016F
:100F70007DE970933400E8958093CA019BBF089582
:100F80002091CF0127FDFCCF9BB78BBFFB01809148
:100F9000CA0123E22093CA010A01E8951124809333
:100FA000CA019BBF0895FC019FB7F894E059FF4F19
:100FB00060958081862380839FBF0895FC019FB741
:100FC000F894E059FF4F8081862B80839FBF08955E
:100FD000E0E7F0E08FEF8193E737F105E1F79FB7A6
:100FE000F894809150008260809350009FBF809160
:100FF000510081FFFCCF80E490E061E00E94C509D0
:101000009FB7F894809150008E7F809350009FBFCF
:101010000895282FAB0186958695869590E0C09619
:10102000277061E070E002C0660F771F2A95E2F733
:1010300025E0880F991F2A95E1F70E9485080895F9
:1010400080E260E073E00E94090881E260E073E002
:101050000E94090882E260E073E00E94090883E2CE
:1010600060E073E00E94090884E260E073E00E949F
:10107000090885E260E073E00E94090886E260E00A
:1010800073E00E94090887E260E073E00E940908AB
:1010900088E268E170E00E94090889E268E170E096
:1010A0000E9409088AE268E170E00E9409088BE268
:1010B00068E170E00E9409088CE268E170E00E943B
:1010C00009088DE268E170E00E9409088EE268E19B
:1010D00070E00E9409088FE268E170E00E94090850
:1010E00083E160E073E00E94090882E160E070E063
:1010F0000E9409088BE160E073E00E9409088AE120
:1011000060E070E00E9409080895CF93DF93DC014E
:10111000FC0120E030E0C62FD0E0CE01022E02C05C
:10112000959587950A94E2F780FD408B2F5F3F4F9E
:1011300031962830310589F750FF0CC051FF04C0AB
:1011400015966C93159703C016966C931697119687
:101150006C9302C012966C93DF91CF9108959B011E
:10116000AC01109200048091010480FDFCCFE0E00E
:10117000F4E020873187CA01AA27BB278093293052
:1011800090932A3085E08093000408959FB7F894E7
:101190002091293030912A3060910804709109041F
:1011A0006115710531F48091030480FF02C02F5F47
:1011B0003F4F9FBF40E050E0A90133272227CB01DA
:1011C000A0E0B0E0282B392B4A2B5B2BB901CA01D8
:1011D00008959B01AC0181E0E0E0F4E0828380911E
:1011E000010480FDFCCFE0E0F4E024873587209304
:1011F0002D3030932E30CA01AA27BB2780932B3085
:1012000090932C308091010480FDFCCF85E0E0E0DC
:10121000F4E082830895E0E0F4E08281869586958B
:1012200080958170089580932F3090933030089589
:101230001F920F920FB60F9208B60F92112418BE8C
:101240008F939F938091293090912A3001968093BB
:10125000293090932A309F918F910F9008BE0F9064
:101260000FBE0F901F9018951F920F920FB60F92FE
:1012700008B60F9209B60F920BB60F92112418BE42
:1012800019BE1BBEEF92FF920F931F932F933F93B4
:101290004F935F936F937F938F939F93AF93BF937E
:1012A000EF93FF932091293030912A3060912B30B9
:1012B00070912C3026173707C0F181E0E0E0F4E0B0
:1012C0008283E0912F30F0913030309771F180912E
:1012D00008049091090440E050E08901FF24EE24C5
:1012E000A0E0B0E0E82AF92A0A2B1B2BCB01A0E0F2
:1012F000B0E0AC013327222780912D3090912E3021
:10130000A0E0B0E0282B392B4A2B5B2B2E153F0594
:101310004007510738F079018A010894E11CF11C5B
:10132000011D111DC801B7011995FF91EF91BF91E2
:10133000AF919F918F917F916F915F914F913F916D
:101340002F911F910F91FF90EF900F900BBE0F9078
:1013500009BE0F9008BE0F900FBE0F901F901895FA
:1013600080E090E064E00E94D30721E0E0E4F0E058
:101370002383E0E0F4E08FEF9FEF8287938710866E
:101380001186228385E0808308951BBEFC0128ED31
:1013900024BF608308951F920F920FB60F9208B674
:1013A0000F9209B60F920BB60F92112418BE19BEF8
:1013B0001BBE2F933F934F935F936F937F938F93B6
:1013C0009F93AF93BF93EF93FF93E0E2F2E04481EA
:1013D0005581E0910330F091043080E092E060E0CC
:1013E0001995FF91EF91BF91AF919F918F917F914F
:1013F0006F915F914F913F912F910F900BBE0F9086
:1014000009BE0F9008BE0F900FBE0F901F90189549
:101410001F920F920FB60F9208B60F9209B60F9255
:101420000BB60F92112418BE19BE1BBE2F933F930B
:101430004F935F936F937F938F939F93AF93BF93DC
:10144000EF93FF93E8E2F2E044815581E0910330AD
:10145000F091043080E092E061E01995FF91EF9106
:10146000BF91AF919F918F917F916F915F914F91BC
:101470003F912F910F900BBE0F9009BE0F9008BEA9
:101480000F900FBE0F901F9018951F920F920FB6DE
:101490000F9208B60F9209B60F920BB60F92112455
:1014A00018BE19BE1BBE2F933F934F935F936F934C
:1014B0007F938F939F93AF93BF93EF93FF93E0E35B
:1014C000F2E044815581E0910330F091043080E0F6
:1014D00092E062E01995FF91EF91BF91AF919F91DA
:1014E0008F917F916F915F914F913F912F910F90CD
:1014F0000BBE0F9009BE0F9008BE0F900FBE0F904D
:101500001F9018951F920F920FB60F9208B60F9268
:1015100009B60F920BB60F92112418BE19BE1BBE4E
:101520002F933F934F935F936F937F938F939F93EB
:10153000AF93BF93EF93FF93E8E3F2E044815581CB
:10154000E0910330F091043080E092E063E019957F
:10155000FF91EF91BF91AF919F918F917F916F918B
:101560005F914F913F912F910F900BBE0F9009BE4D
:101570000F9008BE0F900FBE0F901F9018951F92EE
:101580000F920FB60F9208B60F9209B60F920BB6D4
:101590000F92112418BE19BE1BBE2F933F934F9379
:1015A0005F936F937F938F939F93AF93BF93EF93CB
:1015B000FF93E0E6F2E044815581E0910630F0913E
:1015C000073080E492E060E01995FF91EF91BF91C0
:1015D000AF919F918F917F916F915F914F913F91CB
:1015E0002F910F900BBE0F9009BE0F9008BE0F9069
:1015F0000FBE0F901F9018951F920F920FB60F926B
:1016000008B60F9209B60F920BB60F92112418BEAE
:1016100019BE1BBE2F933F934F935F936F937F939E
:101620008F939F93AF93BF93EF93FF93E8E6F2E01E
:1016300044815581E0910630F091073080E492E0DA
:1016400061E01995FF91EF91BF91AF919F918F91BB
:101650007F916F915F914F913F912F910F900BBEB2
:101660000F9009BE0F9008BE0F900FBE0F901F90F5
:1016700018951F920F920FB60F9208B60F9209B6E7
:101680000F920BB60F92112418BE19BE1BBE2F93DA
:101690003F934F935F936F937F938F939F93AF93FA
:1016A000BF93EF93FF93E0E7F2E044815581E0912F
:1016B0000630F091073080E492E062E01995FF91E6
:1016C000EF91BF91AF919F918F917F916F915F91BA
:1016D0004F913F912F910F900BBE0F9009BE0F902D
:1016E00008BE0F900FBE0F901F9018951F920F927B
:1016F0000FB60F9208B60F9209B60F920BB60F9263
:10170000112418BE19BE1BBE2F933F934F935F93B6
:101710006F937F938F939F93AF93BF93EF93FF93B9
:10172000E8E7F2E044815581E0910630F09107301E
:1017300080E492E063E01995FF91EF91BF91AF9142
:101740009F918F917F916F915F914F913F912F91D9
:101750000F900BBE0F9009BE0F9008BE0F900FBEEA
:101760000F901F90189522E08030920731F48091FD
:101770000230882359F081E008958054924011F09E
:1017800080E0089580910530811181E008952FB7A0
:10179000F89432E08030930729F46093033070931B
:1017A000043007C08054924021F460930630709357
:1017B00007302FBF089522E08030920769F48091AE
:1017C00002308F5F809302308150A9F481E090E075
:1017D00062E00E94D30708958054924061F48091A2
:1017E00005308F5F80930530815029F482E090E0CE
:1017F00062E00E94D3070895FF920F931F938C011C
:10180000FFB6F8940E94DB0BF80180818160808331
:10181000FFBE1F910F91FF90089522E08030920744
:1018200069F4809102308150809302308823A9F4BA
:1018300081E090E062E00E94DE07089580549240CB
:1018400061F480910530815080930530882329F41C
:1018500082E090E062E00E94DE070895DF92EF925E
:10186000FF920F931F93CF93DF938C017A01005E59
:101870001F4FC62FD0E083E0CC0FDD1F8A95E1F724
:10188000C00FD11F00521040DFB6F894C8010E946B
:10189000DB0B8881F70180838A8182838981818340
:1018A000C8010E940D0CDFBEDF91CF911F910F91F7
:1018B000FF90EF90DF900895DF92EF92FF920F93E9
:1018C0001F93CF93DF938C017A01005E1F4FC62FC9
:1018D000D0E093E0CC0FDD1F9A95E1F7C00FD11F48
:1018E00000521040DFB6F894C8010E94DB0BF701EC
:1018F0008081888382818A8381818983C8010E9453
:101900000D0CDFBEDF91CF911F910F91FF90EF90F3
:10191000DF900895DF92EF92FF920F931F938C0157
:101920007B01DFB6F8940E94DB0BF8018081807C9C
:10193000F7018083F801808D918DF701858396836F
:10194000F8018281F7018283F8018481F7018483A1
:10195000F8018381F7018383F8018181F701818395
:10196000C8010E940D0CDFBE1F910F91FF90EF90F8
:10197000DF9008951F93FC011FB7F89480818E7F3C
:101980008083CF010E940D0C1FBF1F9108950F93FC
:101990001F938130910589F08130910528F00297DD
:1019A000A9F020E030E020C082E061E20E94222421
:1019B000182F00E082E060E211C082E065E20E9440
:1019C0002224182F00E082E064E208C082E06FE287
:1019D0000E942224182F00E082E06EE20E9422245E
:1019E000282F30E0202B312BC9011F910F91089532
:1019F000CF92DF92EF92FF921F93CF93DF93EC0190
:101A00007B0182E0C030D80719F480E090E006C086
:101A1000E2E0C034DE0721F581E090E00E94C70CCF
:101A20006C011FB7F894CE010E94DB0B288182E085
:101A30008883CC86DD86F70185819681888F998F92
:101A400082818A8384818C8383818B838181898352
:101A500021708081282B2883CE010E940D0C1FBF8E
:101A6000DF91CF911F91FF90EF90DF90CF9008957D
:101A7000E0910830F0910930878390876187728701
:101A80000895E0910830F091093083879487658745
:101A9000768708959C01E0910A30F0910B3008C0E0
:101AA000808191818217930741F00380F481E02DBA
:101AB0003097B1F72EEF3FEF06C0678370874387FB
:101AC000548720E030E0C90108959C01E0910A307C
:101AD000F0910B3008C0808191818217930741F00B
:101AE0000380F481E02D3097B1F72EEF3FEF06C071
:101AF000618772874587568720E030E0C9010895E5
:101B0000AF92BF92CF92DF92EF92FF920F931F930B
:101B1000DF93CF930F920F92CDB7DEB76C01162FE4
:101B2000072F7A0159011F5F19831150E091083086
:101B3000F0910930228133818481958160E070E0E9
:101B400041E050E0F9011995E0910830F091093039
:101B50002281338184819581BE016F5F7F4F41E097
:101B600050E0F9011995E0910830F0910930208199
:101B7000318184819581BE016E5F7F4F41E050E0ED
:101B8000F90119959A818981A0910830B0910930A5
:101B9000981781F01296ED91FC91139714968D9100
:101BA0009C91159760E070E040E050E0199520EFBF
:101BB0003FEF30C01296ED91FC91139714968D91E2
:101BC0009C911597B601412F502F1995E09108303F
:101BD000F09109302081318184819581B701A5017F
:101BE000F9011995E0910830F09109302281338193
:101BF0008481958160E070E040E050E0F901199542
:101C0000F701808191810E94D417F701808391832D
:101C100020E030E0C9010F900F90CF91DF911F912C
:101C20000F91FF90EF90DF90CF90BF90AF9008950D
:101C3000DF93CF9300D00F92CDB7DEB797E19983B2
:101C40008A83CE01019662E070E0AE014D5F5F4F86
:101C500022E030E00E94800D9C0197FD02C02B81A4
:101C60003C81C9012496CDBFDEBFCF91DF9108959D
:101C70000F931F93DF93CF93CDB7DEB72597CDBFDB
:101C8000DEBF8C018AE18983CE01019661E070E0BC
:101C9000AE014E5F5F4F24E030E00E94800D9C015A
:101CA00097FD05C08D81F80180832A813B81C901A0
:101CB0002596CDBFDEBFCF91DF911F910F91089583
:101CC000DF93CF9300D00F92CDB7DEB796E1998323
:101CD0008A83CE01019662E070E0AE014D5F5F4FF6
:101CE00022E030E00E94800D9C0197FD02C02B8114
:101CF0003C81C9012496CDBFDEBFCF91DF9108950D
:101D00002F923F924F925F926F927F928F929F920B
:101D1000AF92BF92CF92DF92EF92FF920F931F93F9
:101D2000DF93CF93CDB7DEB76997CDBFDEBF5C0140
:101D30004B013A0129011701760189E08983CE011F
:101D4000019661E070E0AE014E5F5F4F28E130E048
:101D50000E94800D9C0197FD52C0A114B10449F06E
:101D60008E819F81A885B985F50180839183A283A7
:101D7000B3838114910449F08A859B85AC85BD8528
:101D8000F40180839183A283B3836114710449F0C9
:101D90008E859F85A889B989F30180839183A28369
:101DA000B3834114510449F08A899B89AC89BD8968
:101DB000F20180839183A283B3830115110539F069
:101DC0008D81992787FD9095F80180839183E11497
:101DD000F10439F08C81992787FD9095F701808374
:101DE00091832114310449F08E899F89A88DB98D82
:101DF000F10180839183A283B3832A813B81C9014E
:101E00006996CDBFDEBFCF91DF911F910F91FF90FB
:101E1000EF90DF90CF90BF90AF909F908F907F908A
:101E20006F905F904F903F902F900895CF92DF92E8
:101E3000EF92FF920F931F938C0180E090E060E09F
:101E400070E040E050E020E030E0EE24FF24CC24BD
:101E5000DD240E94800E1F910F91FF90EF90DF9084
:101E6000CF900895CF92DF92EF92FF920F931F933E
:101E700000E010E0EE24FF24CC24DD240E94800E3C
:101E80001F910F91FF90EF90DF90CF900895DF9317
:101E9000CF9300D00F92CDB7DEB799E199838A83B3
:101EA000CE01019662E070E0AE014D5F5F4F22E02F
:101EB00030E00E94800D9C0197FD02C02B813C8187
:101EC000C9012496CDBFDEBFCF91DF9108950F9356
:101ED000DF93CF93CDB7DEB76697CDBFDEBFFC01F2
:101EE00088E08B83309749F080819181A281B38112
:101EF0008F839887A987BA8704C01F82188619869E
:101F00001A866115710551F0FB0180819181A281D2
:101F1000B3818B879C87AD87BE8704C01B861C86D8
:101F20001D861E864115510551F0FA01808191816F
:101F3000A281B3818F87988BA98BBA8B04C01F862F
:101F4000188A198A1A8A2115310551F0F901808100
:101F50009181A281B3818B8B9C8BAD8BBE8B04C096
:101F60001B8A1C8A1D8A1E8A0E83CE01039664E199
:101F700070E0AE014F5F5F4F22E030E00E94800DC5
:101F80009C0197FD02C029813A81C9016696CDBFA7
:101F9000DEBFCF91DF910F9108950F931F938C01B6
:101FA00080E090E060E070E040E050E020E030E071
:101FB0000E94670F1F910F9108950F931F9300E0E8
:101FC00010E00E94670F1F910F910895DF93CF9348
:101FD00000D0CDB7DEB784E08983CE01019661E001
:101FE00070E0AE014E5F5F4F22E030E00E94800D56
:101FF0009C0197FD02C02A813B81C9012396CDBF78
:10200000DEBFCF91DF910895DF92EF92FF920F93A1
:102010001F93DF93CF93CDB7DEB72597CDBFDEBF3C
:1020200087E78A8388E18983CE01019661E070E0C9
:10203000AE014C5F5F4F22E030E00E94800D9C01BA
:1020400097FD66C0E0910830F0910930228133811C
:102050008481958160E070E041E050E0F9011995DC
:10206000E0910830F091093082E0E82EF12CEC0E7E
:10207000FD1E2281338184819581B70141E050E0CA
:10208000F9011995E0910830F09109308E010D5F4A
:102090001F4F2081318184819581B80141E050E05A
:1020A000F9011995DE2CEF2CF02E012F1BC0129692
:1020B000ED91FC91139714968D919C9115976D2D30
:1020C0007E2D41E050E01995E0910830F091093003
:1020D00020813181848195816F2D702F41E050E006
:1020E000F90119958B81A0910830B09109308E3299
:1020F000F1F21296ED91FC91139714968D919C91AB
:10210000159760E070E040E050E019952C813D812A
:10211000C9012596CDBFDEBFCF91DF911F910F91F1
:10212000FF90EF90DF9008950F931F93DF93CF936D
:10213000CDB7DEB72C97CDBFDEBF8B0125E129835C
:102140000E94D0178B839C83CE01019664E070E0DF
:10215000AE014B5F5F4F28E030E00E94800D9C0194
:1021600097FD0DC02D813E8137FD09C089859A8577
:10217000AB85BC85F80180839183A283B383C901B9
:102180002C96CDBFDEBFCF91DF911F910F910895A7
:10219000AF92BF92CF92DF92EF92FF920F931F9375
:1021A000DF93CF93CDB7DEB72E97CDBFDEBF5B01F8
:1021B0006A01790122E12B830E94D0178D839E83CF
:1021C000C6010E94D0178F839887F7018081918183
:1021D000A281B3818B879C87AD87BE87C8010E948F
:1021E000D01789879A87CE0103966CE070E0AE0124
:1021F0004F5F5F4F22E030E00E94800DAC0197FD01
:1022000016C049815A8157FD12C0C416D5061CF468
:1022100040EF5FEF0CC0E0910830F091093022816F
:10222000338184819581B501F9011995AC01CA0109
:102230002E96CDBFDEBFCF91DF911F910F91FF9002
:10224000EF90DF90CF90BF90AF900895EF92FF9204
:102250000F931F93DF93CF93CDB7DEB72897CDBFF2
:10226000DEBF7B018A0121E12B830E94D0178D8381
:102270009E83C8010E94D0178F839887CE01039652
:1022800066E070E0AE014F5F5F4F22E030E00E94F9
:10229000800DAC0197FD16C049815A8157FD12C0CF
:1022A000041715071CF440EF5FEF0CC0E0910830F5
:1022B000F09109302281338184819581B701F90140
:1022C0001995AC01CA012896CDBFDEBFCF91DF9131
:1022D0001F910F91FF90EF900895EF92FF920F934F
:1022E0001F93DF93CF93CDB7DEB72A97CDBFDEBF65
:1022F0007B018A0120E12D830E94D0178F8398876C
:10230000C8010E94D01789879A87E0910830F09120
:102310000930228133818481958160E070E041E061
:1023200050E0F901199587E08983E0910830F09138
:1023300009302281338184819581BE016F5F7F4F97
:1023400041E050E0F9011995E0910830F091093031
:102350002081318184819581BE016E5F7F4F41E094
:1023600050E0F90119959A818981A0910830B091C6
:1023700009309817E1F01296ED91FC91139714969D
:102380008D919C91159760E070E040E050E01995C8
:10239000E0910830F0910930228133818481958168
:1023A00060E070E040E050E0F90119954BC01296F2
:1023B000ED91FC91139714968D919C911597BE0108
:1023C0006B5F7F4F46E050E01995E0910830F09147
:1023D00009302081318184819581BE016D5F7F4FFD
:1023E00042E050E0F90119958B819C810E94D4173D
:1023F0008B839C839C0197FF11C0E0910830F09182
:102400000930228133818481958160E070E040E071
:1024100050E0F90119950B811C8130C0A091083062
:10242000B09109300817190784F41296ED91FC91C8
:10243000139714968D919C91159760E070E040E0A1
:1024400050E0199500EF1FEF19C0ED91FC91119725
:1024500014968D919C911597B701A90119958C013E
:10246000E0910830F0910930228133818481958197
:1024700060E070E040E050E0F9011995C8012A964B
:10248000CDBFDEBFCF91DF911F910F91FF90EF90F5
:102490000895EF92FF920F931F93DF93CF93CDB7E1
:1024A000DEB72C97CDBFDEBF9C018B017A01E09196
:1024B0000A30F0910B3008C0808191818217930718
:1024C00041F00380F481E02D3097B1F72EEF3FEF1C
:1024D00026C012828EE08B83C9010E94D0178D83A3
:1024E0009E83F80180819181A281B3818F83988737
:1024F000A987BA87C7010E94D0178B879C87CE0116
:1025000003966AE070E0AE014F5F5F4F22E030E07B
:102510000E94800D9C0197FD02C029813A81C9016A
:102520002C96CDBFDEBFCF91DF911F910F91FF9011
:10253000EF9008951F93DF93CF9300D000D0CDB7D5
:10254000DEB7DC01162FE0910A30F0910B3008C0A5
:10255000808191818A179B0741F00380F481E02DEF
:102560003097B1F72EEF3FEF1DC045835683238789
:10257000348712828DE08B83CD010E94D0178D832A
:102580009E831C83CE01039664E070E0AE014F5F32
:102590005F4F22E030E00E94800D9C0197FD02C059
:1025A00029813A81C9012696CDBFDEBFCF91DF9147
:1025B0001F910895EF92FF920F931F93DF93CF9394
:1025C000CDB7DEB72C97CDBFDEBF8B017A012CE0F3
:1025D0002B830E94D0178D839E83F8018081918187
:1025E000A281B3818F839887A987BA87C7010E9488
:1025F000D0178B879C87CE0103966AE070E0AE010E
:102600004F5F5F4F22E030E00E94800D9C0197FDFC
:1026100002C029813A81C9012C96CDBFDEBFCF917E
:10262000DF911F910F91FF90EF900895AF92BF92AD
:10263000CF92DF92EF92FF920F931F93DF93CF938E
:10264000CDB7DEB76597CDBFDEBF809108309091E2
:102650000930892B09F491C185E08983CE01019667
:1026600061E070E0AE014C5F5F4F22E030E00E941D
:10267000800D97FD19C08C819D81009799F4E091A0
:102680000830F0910930278130852115310501F19D
:10269000868180FD1DC0816086838185928561E091
:1026A00070E014C097FF14C0E0910830F091093039
:1026B000278130852115310559F0868180FF08C0BA
:1026C0008E7F86838185928560E070E0F90119959F
:1026D000A6E0AA2EB12CAC0EBD1EC50160E070E0D4
:1026E00040E050E020E030E000E010E0FAE0EF2EC3
:1026F000F12CEC0EFD1EE2E0CE2ED12CCC0EDD1E18
:102700000E94800E0097A1F4E0910830F09109300A
:10271000238534852115310521F1868181FD21C074
:102720008260868385859685B501F901199519C062
:1027300097FF15C0E0910830F0910930238534856A
:102740002115310581F1868181FF2DC08D7F868322
:102750008585968560E070E0F901199524C0892B84
:1027600011F5E0910830F091093027853089211565
:102770003105C9F08A819B81009731F48189928962
:10278000BE01665F7F4F07C08F5F9F4F61F48189F5
:10279000928960E070E0F9011995E0910830F091BC
:1027A00009301786108AE0910830F091093086814F
:1027B0008460868300910A3010910B3033E1B32E90
:1027C0002EE0C22ED12CCC0EDD1E92E1E92EF12C92
:1027D000EC0EFD1E8EC0D8018D919C91BE860E948C
:1027E000D017888B998BC60164E070E0A70124E0C4
:1027F00030E00E94800DAC0197FD22C09D894A897E
:102800005B8957FD1DC09130C9F4F801828180FDBC
:1028100041C00780F085E02D3097E1F181608D7F28
:10282000D80112968C9312976D917C9111971B96FB
:102830008D919C911C9741E050E057C09430B9F4C1
:10284000F801828181FD25C00780F085E02D309759
:1028500001F18E7F8260D80112968C9312976D9150
:102860007C9111971B968D919C911C973CC0933045
:1028700089F4D8011596ED91FC911697309751F097
:102880006D917C9111971B968D919C911C97199538
:102890002DC094E0141615067CF4D8011996ED911C
:1028A000FC911A97309741F06D917C9111971D968C
:1028B0008D919C911E9719C09923C1F4F8018281D2
:1028C00080FF14C00184F285E02D309779F08E7F6F
:1028D000D80112968C9312976D917C9111971D9649
:1028E0008D919C911E9740E050E01995F80103816D
:1028F00014810115110509F06ECFE0910830F091B7
:10290000093086818B7F8683A0910A30B0910B308D
:10291000EE24FF2430C012968C91129782FF23C0C0
:10292000E114F10459F4E0910A30F0910B30838105
:10293000948180930A3090930B3007C013968D9149
:102940009C911497F7018383948313961C9113979A
:1029500014960C911497CD010E94AA46212F302F76
:10296000C901DC0108C07D0113968C911397149660
:102970009C919C01D901109771F66596CDBFDEBF81
:10298000CF91DF911F910F91FF90EF90DF90CF904B
:10299000BF90AF9008950F931F93DF93CF9300D014
:1029A00000D0CDB7DEB78C018FE08B83C8010E94C9
:1029B000D0178D839E83CE01039664E070E0AE0154
:1029C0004F5F5F4F22E030E00E94800D60910A303F
:1029D00070910B30DB0140E050E034C08D919C9150
:1029E00011978017910731F512969C91129792FDDD
:1029F00021C0E0910830F0910930868182FF04C047
:102A0000946012969C9320C04115510541F4FB013E
:102A10008381948180930A3090930B3007C0139682
:102A20008D919C911497FA0183839483CD010E9428
:102A3000AA460AC0AD0113968C91139714969C91E7
:102A40009C01D901109751F680E090E02696CDBF09
:102A5000DEBFCF91DF911F910F910895EF92FF920A
:102A60000F931F93DF93CF93CDB7DEB7C358D040FA
:102A7000CDBFDEBF9C018B017A010097C1F1FC0143
:102A800001900020E9F73197E81BF90BE038F105D8
:102A900070F5E0910830F091093087859089892B95
:102AA00019F022EF3FEF25C08AE08B83CE01049618
:102AB000B9010E947E49CE01039661E870E0AE0143
:102AC0004F5F5F4F22E030E00E94800D9C0197FD38
:102AD00010C029813A812115310559F4E09108305F
:102AE000F09109300787108BE18AF28A02C02EEF3D
:102AF0003FEFC901CD57DF4FCDBFDEBFCF91DF9193
:102B00001F910F91FF90EF900895EF92FF920F9316
:102B10001F93DF93CF9300D000D0CDB7DEB77C01F9
:102B200081E090E06FE070E00E94E1458C01009749
:102B300029F4BDEFEB2EBFEFFB2E3BC084E18B836E
:102B4000C7010E94D0178D839E83CE01039664E057
:102B500070E0AE014F5F5F4F22E030E00E94800DD9
:102B60007C0197FF04C0C8010E94AA4622C0898147
:102B70009A8197FF06C0C8010E94AA46E980FA80A0
:102B800018C0F8018083918313821482828181604E
:102B90008283E0910A30F0910B30CF010380F48101
:102BA000E02D3097D1F7FC0103831483F801E08016
:102BB000F180C7012696CDBFDEBFCF91DF911F9177
:102BC0000F91FF90EF900895EF92FF920F931F9354
:102BD000DF93CF93CDB7DEB72597CDBFDEBF182FDC
:102BE000062F81E090E06FE070E00E94E1457C01FB
:102BF000009719F40DEF1FEF3CC08BE08B831C8313
:102C00000D83CE01039663E070E0AE014F5F5F4F2E
:102C100022E030E00E94800D8C0197FF04C0C701C4
:102C20000E94AA4626C089819A8197FF06C0C701E3
:102C30000E94AA4609811A811CC0F70180839183F2
:102C400013821482E0910A30F0910B30309729F40E
:102C5000E0920A30F0920B3009C0CF010380F4817A
:102C6000E02D3097D1F7FC01E382F482F701008177
:102C70001181C8012596CDBFDEBFCF91DF911F9195
:102C80000F91FF90EF9008950F931F93DF93CF93D1
:102C9000CDB7DEB7E397CDBFDEBF8C0186E0898379
:102CA000CE01019661E070E0AE014E5F5F4F22E31E
:102CB00030E00E94800D9C0197FD16C001151105A2
:102CC00089F0D8019196FE013C9686E001900D9224
:102CD0008150E1F7D801FE01729681E201900D92D8
:102CE0008150E1F72A813B81C901E396CDBFDEBF68
:102CF000CF91DF911F910F9108950F931F93DF9351
:102D0000CF93CDB7DEB7E397CDBFDEBF8C0186E0B2
:102D10008983CE01019661E070E0AE014E5F5F4FA6
:102D200022E330E00E94800D9C0197FD0DC001154B
:102D3000110541F0D801FE01369686E001900D9212
:102D40008150E1F720E030E0C901E396CDBFDEBF5E
:102D5000CF91DF911F910F910895FF920F931F93D1
:102D6000DF93CF930F92CDB7DEB7DB0127E729833F
:102D700061E370E3609308307093093023E1FB0155
:102D800011922A95E9F78093313090933230A093D5
:102D90003330B09334304093353050933630CA01DD
:102DA00060E070E041E050E0FD011995E0910830ED
:102DB000F091093022813381848195818E010F5FEA
:102DC0001F4FB80141E050E0F9011995E09108303A
:102DD000F09109302081318184819581B80141E0F1
:102DE00050E0F9011995F02E012F0CC0ED91FC91E6
:102DF000119714968D919C9115976F2D702F41E02E
:102E000050E019958981A0910830B09109308E3237
:102E100069F31296ED91FC91139714968D919C9104
:102E2000159760E070E040E050E0199580E090E098
:102E30000F90CF91DF911F910F91FF9008951F93F5
:102E4000DF93CF93CDB7DEB7C856D040CDBFDEBF3E
:102E50009C01142F86E6FE013396DF011D928A95B0
:102E6000E9F783E08B832115310541F0DE011796E8
:102E7000F90181E201900D928150E1F76115710530
:102E800031F0CE0188964FE350E00E949349FE0155
:102E9000E859FF4F1083CE01039666E670E0AE015D
:102EA0004F5F5F4F22E030E00E94800D9C0197FD54
:102EB00002C029813A81C901C859DF4FCDBFDEBFA9
:102EC000CF91DF911F910895CF92DF92EF92FF9201
:102ED0000F931F93DF93CF93CDB7DEB76997CDBF25
:102EE000DEBF8C017B016A0182E08983CE010196FD
:102EF00061E070E0AE014E5F5F4F28E130E00E947C
:102F0000800D9C0197FD16C02A813B8137FD12C0C0
:102F10008E819F81A885B985F80180839183A283E2
:102F2000B383C701BE01665F7F4FA6010E9493492C
:102F30002A813B81C9016996CDBFDEBFCF91DF9168
:102F40001F910F91FF90EF90DF90CF9008951F9306
:102F5000DF93CF93CDB7DEB72C97CDBFDEBF142F55
:102F60001D820E94D81769877A878B879C8718876C
:102F7000CE01059668E070E0AE014F5F5F4F24E040
:102F800030E00E94800D9C0197FD02C029813A81AA
:102F9000C9012C96CDBFDEBFCF91DF911F9108955F
:102FA000282F892F922F0895282F892F922F089547
:102FB000EF92FF920F931F93E92EFF240027112712
:102FC000562F442733272227E22AF32A042B152BD6
:102FD0002227362F472F582F207030705070E22A4A
:102FE000F32A042B152B672F782F892F99276070D0
:102FF00080709070E62AF72A082B192BB701C801B8
:103000001F910F91FF90EF9008950E94D817089597
:103010002F923F924F925F926F927F928F929F92E8
:10302000AF92BF92CF92DF92EF92FF920F931F93D6
:10303000DF93CF93CDB7DEB76497CDBFDEBFFC0182
:10304000698B7A8B8081C82EDD24C7FCD0944E0119
:103050000894811C911C9E01235F3F4F2B8B3C8B5E
:103060008C2D80538A3008F048C130E3C316D10458
:1030700021F07AE0672E712C1BC031968081C82E1A
:10308000DD24C7FCD09448E7C416D10441F058E5CC
:10309000C516D10421F068E0662E712C09C0319666
:1030A0008081C82EDD24C7FCD09450E1652E712CA0
:1030B0005F010894A11CB11CEE24FF2487011301B9
:1030C000442437FC4094542CD50111979C2D8C2D11
:1030D00080538A30A0F4C801B701A20191010E9477
:1030E0005245E0EDFFEFCE0EDF1E76010027F7FC24
:1030F0000095102FE60EF71E081F191F2BC0F0E1D8
:103100006F16710489F52C2D2156263048F08C2D30
:103110008154863048F52A3118F021E430E002C0AD
:1031200021E630E0D801C70144E0880F991FAA1FAB
:10313000BB1F4A95D1F74AE050E0C40ED51EC21A13
:10314000D30A76010027F7FC0095102FE82AF92A08
:103150000A2B1B2BF5018081C82EDD24C7FCD094DF
:103160000894A11CB11CB0CFFEE2CF16D104C1F46B
:103170002B893C898216930609F4BFC0F401E082D2
:10318000F1820283138324E030E0820E931EFD015E
:10319000319611968C91C82EDD24C7FCD09460CF57
:1031A000C114D104F1F0903208F4A7C0C7FCA5C047
:1031B00030E2C316D104A9F04CE0C416D10489F062
:1031C0005AE0C516D10469F08DE0C816D10449F063
:1031D00099E0C916D10429F0EBE0CE16D10409F02C
:1031E0008CC0CE0101969401281B390BC90195951D
:1031F00087959595879501968230910571F083307A
:10320000910524F4892B09F478C066C083309105B8
:10321000B9F0049709F060C035C030E0E31630E043
:10322000F30630E0030731E0130708F066C0898138
:103230009A81AB81BC81B82FAA279927882748C0DB
:1032400040E0E41640E0F40641E0040740E01407E3
:1032500008F053C02D813E814F815885A901332745
:10326000222789819A81AB81BC81B82FAA2799270F
:103270008827282B392B4A2B5B2BE22AF32A042B95
:10328000152B2AC05FEFE516F1040105110509F0C1
:10329000A0F58D819E81AF81B885DC0199278827B3
:1032A00029813A814B815C81522F44273327222781
:1032B000822B932BA42BB52B29853A854B855C85D6
:1032C000542F432F322F2227822B932BA42BB52B45
:1032D000E82AF92A0A2B1B2B89899A89892B51F014
:1032E000C801B7010E94D817E989FA896083718300
:1032F0008283938321E030E002C020E030E0C90106
:103300006496CDBFDEBFCF91DF911F910F91FF90EB
:10331000EF90DF90CF90BF90AF909F908F907F9075
:103320006F905F904F903F902F900895AF92BF9213
:10333000CF92DF92EF92FF920F931F93DF93CF9381
:10334000CDB7DEB72797CDBFDEBFFC01808191816D
:10335000A281B3818C839D83AE83BF83F4E0EF2E83
:10336000F12CEC0EFD1E0CE010E36E010894C11C64
:10337000D11C5EE2E7E0AE2EB12CAC0EBD1ED70133
:103380004C9130E0842F6AE00E947145292F842FF0
:103390000E947145482FF601E30FF11D205D208347
:1033A0003F5F882379F7932FF7011082D80106C079
:1033B0003150F601E30FF11D80818D933323C1F766
:1033C000F801E90FF11DDF015D938D01EA14FB04A3
:1033D00021F00894E11CF11CD2CF10828CE090E324
:1033E0002796CDBFDEBFCF91DF911F910F91FF9048
:1033F000EF90DF90CF90BF90AF900895CF93DF9381
:10340000EC01DB0116964D935C931797EA81FB81E3
:10341000309719F46A837B8309C0CF010084F1855A
:10342000E02D3097D1F7FC01A087B18718961D9247
:103430001C921997DF91CF910895FB014683578322
:10344000DC019E966D937C939F970895FC0180818B
:1034500091810895CF92DF92EF92FF920F931F9385
:10346000CF93DF938C016B017A01C0E0D0E012C0F2
:10347000F601EC0FFD1F6081772767FD7095D8017D
:103480001696ED91FC91179718968D919C9119972E
:1034900019952196CE15DF055CF3DF91CF911F9131
:1034A0000F91FF90EF90DF90CF900895CF93DF932F
:1034B000EC01009749F08A859B85009711F00E94E6
:1034C000AA46CE010E94AA46DF91CF9108958F921D
:1034D0009F92AF92BF92CF92DF92EF92FF920F93A3
:1034E0001F93CF93DF934C01162F072F81E090E0BD
:1034F00061E070E00E94E145EC01009709F44AC0E8
:10350000812F902F9C018901CC24DD245401089443
:10351000A108B1083CC0EE24FF24CA14DB041CF44B
:1035200081E0E82EF12CDE010D900020E9F71197E3
:10353000AC1BBD0BF80180819181FC010190002042
:10354000E9F73197E81BF90BAE0FBF1F1196AE0DCF
:10355000BF1DCE01BD010E940247009731F4CE018C
:103560000E94AA46C0E0D0E015C0EC01F8016081DD
:1035700071810E946A49EF2829F0CE0160E070E273
:103580000E946A490894C11CD11C0E5F1F4FC814C9
:10359000D9040CF2CE01DF91CF911F910F91FF90D2
:1035A000EF90DF90CF90BF90AF909F908F90089555
:1035B000CF92DF92EF92FF920F931F93DF93CF93FF
:1035C000CDB7DEB720E1E22EF12CEC0EFD1E80EA35
:1035D00090E00E94FD458C01009779F060EA70E070
:1035E0004E855F8597010E94264A6C0197FD02C0B7
:1035F000780119C0C8010E94AA469DEFC92E9FEF0D
:10360000D92E18C00894E11CF11C772767FD70952E
:10361000AC85BD851696ED91FC91179718968D9106
:103620009C9119971995F7016081662359F7C80194
:103630000E94AA46C601CF91DF911F910F91FF9082
:10364000EF90DF90CF900895EF92FF920F931F932A
:10365000CF93DF938C01DC011296CD91DC9113970F
:1036600033E0E32E30E2F32E24C0288139818C81AF
:103670009D81009711F482E090E2EDB7FEB7389794
:10368000EDBFFEBF3196ADB7BEB711960D931C933B
:103690001297E282F38224833583868397830E9484
:1036A000D81A0884D985C02DEDB7FEB73896EDBF7E
:1036B000FEBF2097D1F6DF91CF911F910F91FF9020
:1036C000EF9008958F929F92AF92BF92CF92DF9228
:1036D000EF92FF920F931F93CF93DF938C016B01B7
:1036E0005A01922E832E6115710511F181E090E04F
:1036F00060E370E00E94E145EC017C010097E9F194
:103700000115110511F40EE010E20C831D8380EA0F
:1037100090E08C879D8781E090E060EA70E00E94F5
:10372000E1458A879B87009731F4CE010E94AA4623
:10373000EE24FF2422C09A8A8B8ACE82DF82A8865A
:10374000B98690FC1AC000D000D0EDB7FEB7319614
:10375000ADB7BEB71196CD93DC93129780E190E29E
:10376000828393838C819D81848395830E94D81A60
:103770008DB79EB706968DBF9EBFC701DF91CF91D3
:103780001F910F91FF90EF90DF90CF90BF90AF907F
:103790009F908F9008952F923F924F925F926F92D9
:1037A0007F928F929F92AF92BF92CF92DF92EF92D1
:1037B000FF920F931F93DF93CF93CDB7DEB7C05522
:1037C000D040CDBFDEBF1C01142F052F29012DB71E
:1037D0003EB7285030402DBF3EBFEDB7FEB7319603
:1037E000ADB7BEB711968D939C93129784E190E28A
:1037F0008283938364837583468257820E94D81A9A
:10380000212F302FC9013C0188249924EDB7FEB740
:103810003896EDBFFEBF4EE2A42E8EC081E090E050
:103820008C0F9D1F800F911FC414D5042CF52DB74C
:103830003EB7285030402DBF3EBFEDB7FEB73196A2
:10384000ADB7BEB711968D939C93129780E590E02B
:10385000801B910B828393832CE230E22483358397
:10386000D7018C91868317820E94D149EDB7FEB7AC
:103870003896EDBFFEBF04C062E370E20E947E494D
:103880000D5F1F4F0894C11CD11C0894E11CF11C52
:103890000033110519F6CE01C19666E370E20E946D
:1038A0007E4963018E010F5C1F4FEE24FF24C70188
:1038B000880D991D841595058CF4D601BC908B2D2F
:1038C00090E00E942D4998012F5F3F4F892B19F0FE
:1038D000F801B08202C0D801AC9289010894E11CC1
:1038E000F11C0894C11CD11CB0E1EB16F104F9F6EF
:1038F000F801108200D000D0EDB7FEB73196ADB719
:10390000BEB711962D923C92129729E330E22283A2
:10391000338381E090E08C0F9D1F848395830E9408
:10392000D81AA0E1B0E08A0E9B1E6A0E7B1EEDB78E
:10393000FEB73696EDBFFEBF841495042CF46401E7
:10394000730100E010E06ACFC05BDF4FCDBFDEBF88
:10395000CF91DF911F910F91FF90EF90DF90CF906B
:10396000BF90AF909F908F907F906F905F904F909F
:103970003F902F9008957F928F929F92AF92BF9227
:10398000CF92DF92EF92FF920F931F93CF93DF932B
:10399000EC01162F88899989892B31F18E859F85B5
:1039A0008F399105F4F46E3659F0623719F06C35A1
:1039B00099F40DC0EA85FB85E80FF91F8DE005C07D
:1039C000EA85FB85E80FF91F8AE0808305C0EA8558
:1039D000FB85E80FF91F60838E859F8501968E8792
:1039E0009F87188A198A2DC16A3099F16B3024F4A7
:1039F000683009F0F2C00DC06D3059F16C3509F036
:103A0000ECC08A8982FF05C081E090E0888B998BA9
:103A100018C18E859F85892B09F413C18A8981FD80
:103A200014C000D00F92ADB7BEB71196CD93DC9302
:103A3000129781E490E213968D939C9314970E94C1
:103A4000D81A0F900F900F900F908E859F85019739
:103A5000F6C0EA85FB858E859F85E80FF91F1082E9
:103A60008A8981FD10C000D00F92EDB7FEB7C183E7
:103A7000D28385E490E2838394830E94D81A0F90C6
:103A80000F900F900F908A859B851C8A1D8A22E0DB
:103A900030E22E8B3F8B11C08C899D890B96FC01E7
:103AA000EE0FFF1FEC0FFD1F208331830A978C8BD5
:103AB0009D8B0C9749F080E090E060E070E20E94FE
:103AC00055499C01009741F7CE88DF88D6017C904C
:103AD0007720B1F10A811B8188249924EE24FF24E8
:103AE00024C0F801A080B180C501B6010E947549CB
:103AF000009721F1D6010D900020E9F71197AC193C
:103B0000BD09C501B601AD010E948549009741F488
:103B1000EF2829F0780151E0852E912C01C0780121
:103B2000D80118960D911C91199701151105C9F628
:103B3000892831F4E114F10419F08701F80104C077
:103B4000EEA5FFA5309779F08681978188839983C8
:103B50006C897D89AE014A5E5F4F0280F381E02D62
:103B6000CE0119951AC07720C1F000D000D0EDB772
:103B7000FEB73196ADB7BEB71196CD93DC931297D1
:103B800088E490E282839383C482D5820E94D81A0B
:103B9000EDB7FEB73696EDBFFEBF1E861F868A893B
:103BA00080FD4FC000D000D0EDB7FEB73196ADB765
:103BB000BEB71196CD93DC93129780E190E2828399
:103BC00093838C819D81848395830E94D81AEDB75D
:103BD000FEB73696EDBFFEBF34C08E859F858F3908
:103BE00091057CF5812F80528F3558F58A8981FDAA
:103BF0001CC000D000D0EDB7FEB73196ADB7BEB750
:103C00001196CD93DC9312978FE590E28283938394
:103C1000812F992787FD9095848395830E94D81AD8
:103C2000EDB7FEB73696EDBFFEBFEA85FB858E8504
:103C30009F85E80FF91F10838E859F8501968E87DB
:103C40009F87DF91CF911F910F91FF90EF90DF90B1
:103C5000CF90BF90AF909F908F907F900895CF921C
:103C6000DF92EF92FF920F931F93DF93CF93CDB725
:103C7000DEB79CE0E92EF12CEC0EFD1EF701C190A1
:103C8000D1907F0180EA90E00E94FD458C01009771
:103C900071F060EA70E0A60197010E94264A6C016B
:103CA00097FD02C078010DC0C8010E94AA468DEFA1
:103CB000C82E8FEFD82E0CC00894E11CF11C0E9476
:103CC0002243F70180818823B9F7C8010E94AA46E0
:103CD000C601CF91DF911F910F91FF90EF90DF9080
:103CE000CF9008952F923F924F925F926F927F9262
:103CF0008F929F92AF92BF92CF92DF92EF92FF92FC
:103D00000F931F93DF93CF93CDB7DEB7C055D0404D
:103D1000CDBFDEBF162F072F2A0100D000D0EDB790
:103D2000FEB731962EE730E2ADB7BEB711962D93B0
:103D30003C93129782839383448355830E942F1E62
:103D4000212F302FC9013C0188249924EDB7FEB7FB
:103D50003696EDBFFEBF31E3232E312C2C0E3D1ED7
:103D60002EE2A22E87C081E090E08C0F9D1F800F75
:103D7000911FC414D5042CF52DB73EB72850304000
:103D80002DBF3EBFEDB7FEB73196ADB7BEB71196AA
:103D90008D939C93129780E590E0801B910B82831A
:103DA000938326E930E224833583D7018C9186837F
:103DB00017820E94D149EDB7FEB73896EDBFFEBF1E
:103DC00004C06CE970E20E947E490D5F1F4F0894A9
:103DD000C11CD11C0894E11CF11C0033110519F61B
:103DE000C10160EA70E20E947E4963018101EE2414
:103DF000FF24C701880D991D841595058CF4D60103
:103E0000BC908B2D90E00E942D4998012F5F3F4F71
:103E1000892B19F0F801B08202C0D801AC92890157
:103E20000894E11CF11C0894C11CD11CB0E1EB16F4
:103E3000F104F9F6F801108200D00F92E3EAF0E203
:103E4000ADB7BEB71196ED93FC93129721E030E029
:103E50002C0F3D1F13962D933C9314970E942F1EF9
:103E600080E190E0880E991E680E791E0F900F90E9
:103E70000F900F90841495042CF46401730100E0FA
:103E800010E071CFC05BDF4FCDBFDEBFCF91DF91C0
:103E90001F910F91FF90EF90DF90CF90BF90AF9068
:103EA0009F908F907F906F905F904F903F902F905A
:103EB000089597FD03C02BEA30E283C0FC0176969B
:103EC000E631F10508F04AC0E650FF4FEE0FFF1F44
:103ED0000590F491E02D199423EB30E272C026ECAA
:103EE00030E26FC026ED30E26CC02CEE30E269C0EB
:103EF0002AEF30E266C028E031E263C026E131E219
:103F000060C025E231E25DC027E331E25AC025E41A
:103F100031E257C02DE531E254C02AE631E251C00A
:103F200023E731E24EC02FE731E24BC024E831E213
:103F300048C02DE831E245C02CE931E242C024EA14
:103F400031E23FC02CEA31E23CC02FEB31E239C014
:103F50002AEC31E236C022ED31E233C00F920F92EB
:103F600081EE91E2ADB7BEB711968D939C931297F7
:103F70000E942F1EEDB7FEB73897EDBFFEBF3196FA
:103F80008CEF91E2ADB7BEB711968D939C931297CB
:103F90008FE092E28283938388E390E08483958329
:103FA00085E99FE28683978386E392E28087918703
:103FB0000E942F1E28E332E2EDB7FEB73A96EDBF1E
:103FC000FEBFC90108959C01E0911C30F0911D30A5
:103FD00082819381D90118968D939C93199784813E
:103FE0009581FC016E9FC0016F9F900D7E9F900D8B
:103FF000112468EE73E00E947D45D9011A966D93F5
:104000007C931B9716968D919C9117978E7F169691
:104010008D939C9317970895E0911C30F0911D307B
:10402000228133816481758188EE93E0AC01249F05
:10403000C001259F900D349F900D11240E947D4555
:10404000CB010895E0911C30F0911D30309729F09C
:10405000828193810196828393830895CF93DF9326
:10406000C0911C30D0911D30EA81FB812C813D81B3
:10407000AC01429FC001439F900D529F900D1124AF
:1040800068EE73E00E947D456E0F7F1F8A819B81E1
:1040900086179707D8F3DF91CF91089568177907AE
:1040A00058F020E0681B790B6417750708F421E0CD
:1040B00081E0822790E0089520E030E0809590959F
:1040C000860F971F8417950710F021E030E0C90193
:1040D00008956817790730F49C0120953095260FD4
:1040E000371F03C09B01281B390BC9010895EF92AC
:1040F000FF920F931F93CF93DF93E0911C30F091C9
:104100001D3086819781816086839783C081D181AC
:1041100088EEE82E83E0F82E38C00E811F8100FD66
:1041200031C002FD2FC0E0911C30F0911D30628142
:1041300073814A855B85888599850E944E20892BED
:1041400009F101600E831F836C817D81EA81FB810F
:10415000CE0119958E8181FF15C08A859B85E091DE
:104160001C30F0911D30648175819C012E9DC00131
:104170002F9D900D3E9D900D11240E947D45CE01F6
:104180000E94E31F0990D881C02D209731F6E0915D
:104190001C30F0911D30868197818E7F86839783B6
:1041A000C081D181EE24FF2423C08E8182FF1BC0F9
:1041B000E114F10449F4E0911C30F0911D30A0812C
:1041C000B1818D919C9103C088819981F701808391
:1041D000918318810981CE010E94AA46212F302F98
:1041E000C901EC0105C07E01888199819C01E9012A
:1041F0002097D9F6DF91CF911F910F91FF90EF900B
:104200000895CF93DF93EC01009709F442C08E81AB
:1042100082FF31C00F920F9280E492E2ADB7BEB739
:1042200011968D939C9312970E942F1EEDB7FEB7A7
:104230003897EDBFFEBF31968BE592E2ADB7BEB7C2
:1042400011968D939C9312978EE692E282839383CC
:104250008AE690E0848395838FE99FE28683978343
:1042600087E992E2808791870E942F1EEDB7FEB703
:104270003A96EDBFFEBFA0911C30B0911D3016964E
:104280008C91169780FF08C08E819F8184608E83F9
:104290009F8320E030E023C04D915C9111979A01FB
:1042A000E0E0F0E017C02C173D0781F4309731F4BF
:1042B000FA01808191818D939C9304C088819981BA
:1042C00080839183CE010E94AA46E3CFF9018081C9
:1042D00091819C012115310531F72EEF3FEFC90186
:1042E000DF91CF910895AF92BF92CF92DF92EF927C
:1042F000FF920F931F93CF93DF935C016B01EA0151
:1043000079014115510519F400E010E035C081E054
:1043100090E06CE070E00E94E145DC018C010097C8
:1043200059F11296CD93DC9313971496ED92FC926B
:104330001597CD2849F016968D919C91179782601C
:1043400016968D939C931797C0911C30D0911D3079
:10435000E881F981309719F4A883B98309C0CF01A6
:104360000190F081E02D3097D1F7FC01A083B1835B
:10437000CD01B5010E94E31FC801DF91CF911F91CC
:104380000F91FF90EF90DF90CF90BF90AF90089586
:10439000CF93DF93EC01009719F42EEF3FEF14C099
:1043A00081E090E068E070E00E94E145FC018093CC
:1043B0001C3090931D30009719F42DEF3FEF04C08F
:1043C000C483D58320E030E0C901DF91CF91089507
:1043D000CF92DF92EF92FF920F931F93CF93DF93D1
:1043E000F801EC0188E0C03AD807D9F4403885E2FA
:1043F000580780E0680780E0780709F066C0283039
:10440000310509F062C081E0E816F10409F05DC0F1
:104410000115110509F059C0CD2809F056C013E067
:1044200029C0CD2809F051C027303105A1F028302E
:10443000310520F42630310561F407C028303105FC
:1044400031F02930310529F408C011E007C013E02C
:1044500005C010E003C012E001C017E0E130F10533
:1044600031F0E130F10530F0329779F502C0106299
:1044700001C0106382E0E816F10409F418609A01A3
:10448000AB0184E0220F331F441F551F8A95D1F7DB
:10449000213088E4380788EE480781E0580720F08B
:1044A0008CE12FEF3FEF09C060E078E488EE91E007
:1044B0000E94A4452150304088E11C821D832E8338
:1044C0003F838C8320E030E002C026EF3FEFC9013C
:1044D000DF91CF911F910F91FF90EF90DF90CF90E0
:1044E0000895FC01818185FFFDCF6083E05AF8408B
:1044F00071F48091A10886FFFCCF8091A1088064AF
:10450000E0EAF8E0818388EE93E00197F1F70895FF
:10451000DC0120E030E00CC011968C91119787FFF0
:10452000FBCF8C91FB01E20FF31F80832F5F3F4F86
:10453000241735078CF3CA010895CF92DF92EF92CA
:10454000FF920F931F93CF93DF936C017B018A013E
:104550006115710519F0C0E0D0E019C04115510591
:1045600039F08FB7F89480931E3000E010E012C04D
:1045700080911E308FBF0EC0F701EC0FFD1F6081D0
:10458000772767FD7095C6010E9471222196C0179A
:10459000D10794F3C801DF91CF911F910F91FF9044
:1045A000EF90DF90CF900895FC01218130E02078DA
:1045B0003070C901089582309105A1F083309105D2
:1045C00028F4009761F00197B1F406C0833091059B
:1045D00061F0049781F40CC023EB32E23FC025EB7D
:1045E00032E23CC027EB32E239C029EB32E236C07E
:1045F0002BEB32E233C00F920F928DEB92E2ADB70C
:10460000BEB711968D939C9312970E942F1EEDB703
:10461000FEB73897EDBFFEBF319688ED92E2ADB799
:10462000BEB711968D939C9312978BEE92E2828384
:1046300093838BED90E0848395838DEA9FE286835C
:10464000978389E193E2808791870E942F1E2BE157
:1046500033E2EDB7FEB73A96EDBFFEBFC90108954C
:10466000EF92FF920F931F93182F092F7B010E9447
:104670000C20E12FF02FEF2819F006EF1FEF06C0F6
:10468000818187FFFDCF8081082F10E0C8011F9135
:104690000F91FF90EF90089560931F30709320303A
:1046A0000E94B0098DE593E20E9413090E94C6089A
:1046B0000E94E90880E090E00895E0911F30F091B9
:1046C0002030309709F019950E94C6080E94E90829
:1046D00008959C01883091054CF481E090E002C07F
:1046E000880F991F2A95E2F780938706089587E03F
:1046F000E0EAF0E082830E94E8070E94200883E05D
:1047000090E060E10E94D30784E090E060E10E94C5
:10471000D307789480E090E0089520912330309181
:10472000243021513140C9010895FF920F931F9306
:104730008C01F62E60E070E0CB01BA0126E631E094
:1047400040E050E00E9452452091213030912230CB
:1047500040E050E00E94A445209323303093243061
:104760003FB7F894F801208181E090E002C0880F03
:10477000991FFA94E2F7880F880F822B80833FBF3E
:104780001F910F91FF9008950F931F93DF93CF9385
:10479000CDB7DEB72A97CDBFDEBFFE01349687E0E6
:1047A000DF011D928A95E9F78E010F5F1F4F83E0AD
:1047B000D8011D928A95E9F72D819E819F7C86E024
:1047C0008887217E2D831F8291609E8380E092E006
:1047D000BF010E94F80C80E092E065E973E20E945C
:1047E000C70B19821A828B81807F81608B8380E066
:1047F00092E060E0A8010E945C0C82E06FE20E94FF
:104800002224182F00E082E06EE20E94222490E031
:10481000082B192B009321301093223080E092E076
:104820000E94FC0B9FB7F894E0E0F2E08081846086
:1048300080839FBF2A96CDBFDEBFCF91DF911F91AE
:104840000F9108954091CA01E62FFF278093CA0176
:1048500084914093CA0108958F929F92AF92BF9224
:10486000CF92DF92EF92FF920F931F934C0162E081
:1048700072E081E090E00E94D8170E9405185B0169
:104880006C0162E072E081E090E00E94D8170E9423
:1048900005187B018C0162E072E081E090E00E94EB
:1048A000D8170E9405182DB73EB72A5030402DBFAB
:1048B0003EBFEDB7FEB73196ADB7BEB711968D923C
:1048C0009C9212972CE133E2228333835601CC244D
:1048D000DD24BFEFAB22BB24A482B582EF2CF02EE7
:1048E000012F11272FEFE222FF24E682F78270705A
:1048F000608771870E94D81A8DB79EB70A968DBFC0
:104900009EBF1F910F91FF90EF90DF90CF90BF90CF
:10491000AF909F908F9008952DB73EB728503040AC
:104920002DBF3EBFEDB7FEB73196ADB7BEB71196FE
:104930008D939C9312978FE293E282839383648397
:104940007583468357830E94D81A2DB73EB7285FD8
:104950003F4F2DBF3EBF08958F929F92AF92BF925F
:10496000CF92DF92EF92FF920F931F93DF93CF933B
:10497000CDB7DEB76497CDBFDEBF4C01CE01019647
:10498000BE016B5F7F4F40E150E00E9464178C01D5
:1049900097FF05C050E5E52E53E2F52E04C044E52F
:1049A000E42E43E2F42EC8010E94591F2DB73EB7F2
:1049B0002A5030402DBF3EBFEDB7FEB73196ADB7A0
:1049C000BEB711968D929C92129727E533E222830F
:1049D0003383E482F58206831783808791870E9460
:1049E000D81A2DB73EB7265F3F4F2DBF3EBF698116
:1049F0007A818B819C810E9405185B016C01698121
:104A00007A818B819C810E9405187B018C016981D0
:104A10007A818B819C810E940518ADB7BEB71C9727
:104A2000ADBFBEBFEDB7FEB7319611968D929C9289
:104A3000129724E633E2228333835601CC24DD240B
:104A4000BFEFAB22BB24A482B582EF2CF02E012F46
:104A500011272FEFE222FF24E682F7827070608731
:104A60007187CE010596828793870E94D81A8DB7E9
:104A70009EB70C968DBF9EBF6496CDBFDEBFCF9113
:104A8000DF911F910F91FF90EF90DF90CF90BF903B
:104A9000AF909F908F900895EF92FF920F931F9386
:104AA000CF93DF938C01FA0162307105BCF18281F2
:104AB000938169EA75E2A8010E942E15EC0197FF27
:104AC00005C070E5E72E73E2F72E04C064E5E62E1C
:104AD00063E2F62ECE010E94591F2DB73EB72A5031
:104AE00030402DBF3EBFEDB7FEB73196ADB7BEB774
:104AF00011960D931C93129727E533E2228333839B
:104B0000E482F582C683D783808791870E94D81A72
:104B1000EDB7FEB73A96EDBFFEBF14C000D00F92BE
:104B2000ADB7BEB711968D939C93129780E893E230
:104B300013968D939C9314970E94D81A0F900F9000
:104B40000F900F90DF91CF911F910F91FF90EF90F9
:104B500008950F931F93182F092F61157105A9F45C
:104B600000D00F92EDB7FEB73196ADB7BEB7119634
:104B70008C93918382EA93E2828393830E94D81A72
:104B80000F900F900F900F901AC0CB010E949619B2
:104B900000D000D0EDB7FEB73196ADB7BEB71196D5
:104BA0001C9301832EEB33E222833383848395832A
:104BB0000E94D81A8DB79EB706968DBF9EBF1F91D3
:104BC0000F910895EF92FF920F931F93DF93CF936E
:104BD0000F920F92CDB7DEB77C018B01BE016F5FE4
:104BE0007F4F40E050E00E94DE47F8016083718310
:104BF00020E030E089819A818E159F0511F021E037
:104C000030E0C9010F900F90CF91DF911F910F916C
:104C1000FF90EF900895CF92DF92EF92FF920F9363
:104C20001F93DF93CF9300D000D0CDB7DEB76C01D8
:104C3000FA01623071050CF45DC082819381BE017E
:104C40006F5F7F4F0E94E225892B09F453C0898151
:104C50009A81BE016D5F7F4F0E9494108C0197FF77
:104C600005C0F0E5EF2EF3E2FF2E04C0E4E5EE2EE2
:104C7000E3E2FE2EC8010E94591F2DB73EB72A500D
:104C800030402DBF3EBFEDB7FEB73196ADB7BEB7D2
:104C90001196CD92DC92129720ED33E2228333837A
:104CA000E482F58206831783808791870E94D81A51
:104CB000EDB7FEB73A96EDBFFEBFCE0103960E9458
:104CC000961900D000D0EDB7FEB73196ADB7BEB79C
:104CD0001196CD92DC9212972CED33E2228333832E
:104CE000848395830E94D81AEDB7FEB73696EDBF40
:104CF000FEBF14C000D00F92ADB7BEB71196CD92D3
:104D0000DC92129786EE93E213968D939C93149700
:104D10000E94D81A0F900F900F900F902696CDBF3B
:104D2000DEBFCF91DF911F910F91FF90EF90DF9049
:104D3000CF9008952F923F924F925F926F927F9201
:104D40008F929F92AF92BF92CF92DF92EF92FF929B
:104D50000F931F93DF93CF93CDB7DEB72A97CDBFC5
:104D6000DEBF3C016B017A01643071050CF4E1C0D7
:104D7000DA0112968D919C911397BE016F5F7F4F60
:104D80000E94E225892B09F4D4C005E0402E512C65
:104D90004C0E5D1EF70184819581B2010E940818B6
:104DA000892B09F4C6C0D70116960D911C9117974F
:104DB000C801BE016D5F7F4F40E050E00E94DE47BA
:104DC0009B01AC018B819C818017910709F4B1C0D4
:104DD000122F032F37FDADC0E8E0F0E0EE0EFF1E0E
:104DE000C6010497B7010E94671A4C01009709F4A5
:104DF00076C019870A87DC010D900020E9F77D0154
:104E00000894E108F108E81AF90AC2010E9496190B
:104E1000EDB7FEB73A97EDBFFEBF3196ADB7BEB75F
:104E200011966D927C92129725E034E222833383AF
:104E3000E482F58286839783108701870E94D81ABF
:104E4000AA24BB24EDB7FEB73A96EDBFFEBF120110
:104E500011E2412E14E2512E35C06701CA18DB0859
:104E6000B4016A0D7B1D89819A81A6019101098592
:104E70001A850E94C8108C0197FF04C0C4010E94CB
:104E8000AA462FC02DB73EB7285030402DBF3EBF99
:104E9000EDB7FEB73196ADB7BEB711966D927C9265
:104EA00012974282538284839583C81AD90AC68294
:104EB000D7820E94D81AA00EB11EEDB7FEB7389661
:104EC000EDBFFEBFAE14BF0444F2C4010E94AA4667
:104ED000B4E5EB2EB3E2FB2E00E010E006C00DEFD0
:104EE0001FEFA0E5EA2EA3E2FA2EC8010E94591F87
:104EF0002DB73EB72A5030402DBF3EBFEDB7FEB7AD
:104F00003196ADB7BEB711966D927C92129727E598
:104F100033E222833383E482F5820683178380871A
:104F200091870E94D81AEDB7FEB73A96EDBFFEBF43
:104F300014C000D00F92ADB7BEB711966D927C929F
:104F4000129786E394E213968D939C9314970E9494
:104F5000D81A0F900F900F900F902A96CDBFDEBFFA
:104F6000CF91DF911F910F91FF90EF90DF90CF9045
:104F7000BF90AF909F908F907F906F905F904F9079
:104F80003F902F9008954F925F926F927F928F92F1
:104F90009F92AF92BF92CF92DF92EF92FF920F93C8
:104FA0001F93DF93CF930F920F92CDB7DEB73C01E3
:104FB0007B018A01633071050CF4AAC0DA011296F4
:104FC0008D919C911397BE016F5F7F4F0E94E225E8
:104FD000892B09F49DC00C5F1F4FC7010297B801D0
:104FE0000E94671A4C01009709F468C0DC010D901B
:104FF0000020E9F77D010894E108F108E81AF90AB0
:1050000000D000D0EDB7FEB73196ADB7BEB7119660
:105010006D927C92129786E694E282839383E48277
:10502000F5820E94D81AAA24BB24EDB7FEB73696A3
:10503000EDBFFEBF21E2422E24E2522E32C06701B4
:10504000CA18DB08B4016A0D7B1D89819A81A6010B
:105050000E9426118C0197FF04C0C4010E94AA4639
:105060002FC02DB73EB7285030402DBF3EBFEDB703
:10507000FEB73196ADB7BEB711966D927C9212977E
:105080004282538284839583C81AD90AC682D78202
:105090000E94D81AA00EB11EEDB7FEB73896EDBF2C
:1050A000FEBFAE14BF045CF2C4010E94AA4694E5A0
:1050B000E92E93E2F92E00E010E006C00DEF1FEF9D
:1050C00080E5E82E83E2F82EC8010E94591F2DB713
:1050D0003EB72A5030402DBF3EBFEDB7FEB73196E8
:1050E000ADB7BEB711966D927C92129727E533E269
:1050F00022833383E482F582068317838087918736
:105100000E94D81AEDB7FEB73A96EDBFFEBF14C0A5
:1051100000D00F92ADB7BEB711966D927C921297E8
:1051200089E794E213968D939C9314970E94D81A62
:105130000F900F900F900F900F900F90CF91DF91E5
:105140001F910F91FF90EF90DF90CF90BF90AF90A5
:105150009F908F907F906F905F904F900895CF9227
:10516000DF92EF92FF920F931F93DF93CF930F92F3
:105170000F92CDB7DEB76C01FA0162307105ECF128
:1051800082819381BE016F5F7F4F0E94E225892B50
:10519000A1F189819A810E94CB148C0197FF05C0EF
:1051A00040E5E42E43E2F42E04C034E5E32E33E27E
:1051B000F32EC8010E94591F2DB73EB72A50304028
:1051C0002DBF3EBFEDB7FEB73196ADB7BEB7119656
:1051D000CD92DC92129727E533E222833383E48277
:1051E000F58206831783808791870E94D81AEDB7CE
:1051F000FEB73A96EDBFFEBF14C000D00F92ADB718
:10520000BEB71196CD92DC9212978BE994E2139679
:105210008D939C9314970E94D81A0F900F900F9023
:105220000F900F900F90CF91DF911F910F91FF90F2
:10523000EF90DF90CF900895CF92DF92EF92FF92A0
:105240000F931F93DF93CF93CDB7DEB72897CDBFD2
:10525000DEBF6C018A01643071050CF464C0DA01B0
:1052600012968D919C911397BE016F5F7F4F0E94A4
:10527000E225892B09F457C075E0E72EF12CEC0EDE
:10528000FD1EF80184819581B7010E940818892BC1
:1052900009F449C0D80116960D911C911797C801C1
:1052A000BE016D5F7F4F40E050E00E94DE479B01F2
:1052B000AC018B819C8180179107A9F137FD33C028
:1052C00089819A81B701A9010E9449128C0197FF37
:1052D00005C060E5E62E63E2F62E04C054E5E52E37
:1052E00053E2F52EC8010E94591FEDB7FEB73A9759
:1052F000EDBFFEBF3196ADB7BEB71196CD92DC9231
:10530000129727E533E222833383E482F582068312
:105310001783808791870E94D81AEDB7FEB73A9617
:10532000EDBFFEBF14C000D00F92ADB7BEB711964F
:10533000CD92DC92129783EB94E213968D939C931B
:1053400014970E94D81A0F900F900F900F902896E4
:10535000CDBFDEBFCF91DF911F910F91FF90EF90F6
:10536000DF90CF900895CF92DF92EF92FF920F934C
:105370001F93DF93CF9300D00F92CDB7DEB76C01B0
:105380008B017A0181E090E08B839C836230710510
:105390000CF453C0DA0112968D919C911397BE01C3
:1053A0006F5F7F4F0E94E225892B09F446C00230CF
:1053B000110551F0F70184819581BE016D5F7F4F2A
:1053C0000E94E225892BC9F16B817C8189819A81B8
:1053D0004DE35AE296010E949A128C0197FF05C094
:1053E000F0E5EF2EF3E2FF2E04C0E4E5EE2EE3E25B
:1053F000FE2EC8010E94591F2DB73EB72A503040DB
:105400002DBF3EBFEDB7FEB73196ADB7BEB7119613
:10541000CD92DC92129727E533E222833383E48234
:10542000F58206831783808791870E94D81AEDB78B
:10543000FEB73A96EDBFFEBF14C000D00F92ADB7D5
:10544000BEB71196CD92DC92129789ED94E2139635
:105450008D939C9314970E94D81A0F900F900F90E1
:105460000F902496CDBFDEBFCF91DF911F910F919A
:10547000FF90EF90DF90CF900895EF92FF920F93FF
:105480001F93CF93DF93F82EE92E8B0100D000D02D
:10549000EDB7FEB73196ADB7BEB711968C93918339
:1054A0008CEF94E282839383648375830E94D81A7D
:1054B0002DB73EB72A5F3F4F2DBF3EBFC8010E94A8
:1054C0008515EC011816190674F46CE874E24F2D7A
:1054D0005E2D0E944A0DCE0161EA7AE24F2D5E2DCB
:1054E0000E94650D05C0009719F000E513E202C0A7
:1054F00004E513E2CE010E94591FADB7BEB71A975B
:10550000ADBFBEBFEDB7FEB731961196FC92E182FA
:1055100027E533E22283338304831583C683D7834D
:10552000808791870E94D81A2DB73EB7265F3F4FDC
:105530002DBF3EBFDF91CF911F910F91FF90EF9054
:105540000895AF92BF92CF92DF92EF92FF920F93A6
:105550001F93DF93CF93CDB7DEB7C054D040CDBFFC
:10556000DEBF5C017B018A014115510519F420E27F
:1055700035E202C022E335E28DB79EB70A978DBFB0
:105580009EBFEDB7FEB73196ADB7BEB71196AC92E0
:10559000B18283E395E282839383E482F58206837A
:1055A0001783208731870E94D81A8DB79EB70A9635
:1055B0008DBF9EBF6E010894C11CD11C17C0013461
:1055C000110510F4A80102C040E450E0C701B60183
:1055D0000E946D119C01181619068CF7081B190BF7
:1055E000C50161E575E2A6010E94CB1B10161106EC
:1055F00034F3C05CDF4FCDBFDEBFCF91DF911F9191
:105600000F91FF90EF90DF90CF90BF90AF900895F3
:10561000CF92DF92EF92FF920F931F93DF93CF937E
:10562000CDB7DEB72897CDBFDEBF6C018A016430ED
:1056300071050CF464C0DA0112968D919C91139758
:10564000BE016F5F7F4F0E94E225892B09F457C08E
:1056500085E0E82EF12CEC0EFD1EF8018481958189
:10566000B7010E940818892B09F449C0D801169681
:105670000D911C911797C801BE016D5F7F4F40E0EF
:1056800050E00E94DE479B01AC018B819C8180171A
:105690009107A9F137FD33C089819A81B701A9012A
:1056A0000E94DA128C0197FF05C0B0E5EB2EB3E241
:1056B000FB2E04C0A4E5EA2EA3E2FA2EC8010E9444
:1056C000591FEDB7FEB73A97EDBFFEBF3196ADB7A4
:1056D000BEB71196CD92DC92129727E533E2228372
:1056E0003383E482F58206831783808791870E9443
:1056F000D81AEDB7FEB73A96EDBFFEBF14C000D082
:105700000F92ADB7BEB71196CD92DC92129784E599
:1057100095E213968D939C9314970E94D81A0F903C
:105720000F900F900F902896CDBFDEBFCF91DF91E5
:105730001F910F91FF90EF90DF90CF900895AF925F
:10574000BF92CF92DF92EF92FF920F931F93DF935E
:10575000CF930F920F92CDB7DEB76C017B015A0148
:1057600019821A82623071050CF472C0DA01129645
:105770000D911C911397C80167E775E20E94754966
:10578000009719F400E010E014C0C8016EE775E25C
:105790000E947549009719F401E010E00AC0C801A1
:1057A00064E875E20E947549009709F051C002E073
:1057B00010E0B2E0EB16F10459F0F5018481958117
:1057C000BE016F5F7F4F0E94E225892B09F440C024
:1057D00069817A81C8010E94E4158C016CE874E249
:1057E000A6010E944A0DC80161EA7AE2A6010E9460
:1057F000650D17FF05C020E5E22E23E2F22E04C05E
:1058000094E5E92E93E2F92EC8010E94591F2DB7A5
:105810003EB72A5030402DBF3EBFEDB7FEB73196A0
:10582000ADB7BEB71196CD92DC92129727E533E261
:1058300022833383E482F5820683178380879187EE
:105840000E94D81AEDB7FEB73A96EDBFFEBF14C05E
:1058500000D00F92ADB7BEB71196CD92DC921297E1
:1058600088E895E213968D939C9314970E94D81A1A
:105870000F900F900F900F900F900F90CF91DF919E
:105880001F910F91FF90EF90DF90CF90BF90AF905E
:105890000895CF92DF92EF92FF920F931F93DF93C1
:1058A000CF930F920F92CDB7DEB76C01FA01623041
:1058B0007105ECF182819381BE016F5F7F4F0E9481
:1058C000E225892BA1F189819A810E94470F8C01E1
:1058D00097FF05C040E5E42E43E2F42E04C034E512
:1058E000E32E33E2F32EC8010E94591F2DB73EB7B5
:1058F0002A5030402DBF3EBFEDB7FEB73196ADB751
:10590000BEB71196CD92DC92129727E533E222833F
:105910003383E482F58206831783808791870E9410
:10592000D81AEDB7FEB73A96EDBFFEBF14C000D04F
:105930000F92ADB7BEB71196CD92DC92129786EB5F
:1059400095E213968D939C9314970E94D81A0F900A
:105950000F900F900F900F900F90CF91DF911F91AC
:105960000F91FF90EF90DF90CF9008950F931F93CA
:10597000DF93CF930F920F92CDB7DEB78C01CE019C
:1059800001960E94160FAC0197FF03C020E533E299
:1059900002C024E533E28DB79EB70A978DBF9EBF44
:1059A000EDB7FEB73196ADB7BEB711960D931C9308
:1059B00012978FEC95E28283938324833583468309
:1059C000578389819A81808791870E94D81A8DB7E1
:1059D0009EB70A968DBF9EBF0F900F90CF91DF911B
:1059E0001F910F910895CF92DF92EF92FF920F9344
:1059F0001F93DF93CF930F920F92CDB7DEB76C0159
:105A0000FA0162307105ECF182819381BE016F5F12
:105A10007F4F0E94E225892BA1F189819A810E9402
:105A2000CD0F8C0197FF05C060E5E62E63E2F62EF0
:105A300004C054E5E52E53E2F52EC8010E94591F1B
:105A40002DB73EB72A5030402DBF3EBFEDB7FEB751
:105A50003196ADB7BEB71196CD92DC92129727E57D
:105A600033E222833383E482F582068317838087BF
:105A700091870E94D81AEDB7FEB73A96EDBFFEBFE8
:105A800014C000D00F92ADB7BEB71196CD92DC9284
:105A9000129784EE95E213968D939C9314970E942F
:105AA000D81A0F900F900F900F900F900F90CF91EA
:105AB000DF911F910F91FF90EF90DF90CF900895AD
:105AC0000F931F93DF93CF93CDB7DEB76097CDBF12
:105AD000DEBF8C01CE010196BE016B5F7F4FAE0130
:105AE000475F5F4F9E01235F3F4F0E94320FAC0123
:105AF00097FF03C020E533E202C024E533E28DB70F
:105B00009EB708978DBF9EBFEDB7FEB73196ADB774
:105B1000BEB711960D931C9312978CEF95E282837A
:105B2000938324833583468357830E94D81A8DB785
:105B30009EB708968DBF9EBFCE0101960E94961912
:105B400000D000D0EDB7FEB73196ADB7BEB7119615
:105B50000D931C93129724E036E2228333838483CF
:105B600095830E94D81A8DB79EB706968DBF9EBFAB
:105B7000CE0105960E94961900D000D0EDB7FEB771
:105B80003196ADB7BEB711960D931C9312972BE0CB
:105B900036E222833383848395830E94D81A8DB79B
:105BA0009EB706968DBF9EBFCE0109960E9496199C
:105BB00000D000D0EDB7FEB73196ADB7BEB71196A5
:105BC0000D931C93129724E136E22283338384835E
:105BD00095830E94D81A8DB79EB706968DBF9EBF3B
:105BE000CE010D960E94961900D000D0EDB7FEB7F9
:105BF0003196ADB7BEB711960D931C9312972BE15A
:105C000036E222833383848395830E94D81A8DB72A
:105C10009EB706968DBF9EBF6096CDBFDEBFCF916B
:105C2000DF911F910F910895CF92DF92EF92FF9233
:105C30000F931F93DF93CF93CDB7DEB76097CDBFA0
:105C4000DEBF6C018B017A0180918D2F90918E2F98
:105C5000A0918F2FB091902F8D839E83AF83B887B3
:105C600089879A87AB87BC878D879E87AF87B88BDC
:105C7000623071050CF475C0DA0112968D919C9119
:105C80001397BE016F5F7F4F0E940818892B09F49C
:105C900068C00230110541F1F70184819581BE0190
:105CA0006B5F7F4F0E940818892B09F45AC003309C
:105CB0001105D1F0D70116968D919C911797BE01D1
:105CC000675F7F4F0E940818892B09F44AC005308E
:105CD000110554F0F70180859185BE01635F7F4F08
:105CE0000E940818892BE9F1CE010196BE016B5F75
:105CF0007F4FAE01475F5F4F9E01235F3F4F0E9482
:105D0000DD0F8C0197FF05C0E0E5EE2EE3E2FE2EED
:105D100004C074E5E72E73E2F72EC8010E94591FF4
:105D20002DB73EB72A5030402DBF3EBFEDB7FEB76E
:105D30003196ADB7BEB71196CD92DC92129727E59A
:105D400033E222833383E482F582068317838087DC
:105D500091870E94D81AEDB7FEB73A96EDBFFEBF05
:105D600014C000D00F92ADB7BEB71196CD92DC92A1
:105D7000129785E296E213968D939C9314970E9456
:105D8000D81A0F900F900F900F906096CDBFDEBF86
:105D9000CF91DF911F910F91FF90EF90DF90CF9007
:105DA00008958F929F92AF92BF92CF92DF92EF921F
:105DB000FF920F931F93DF93CF93CDB7DEB7C854F5
:105DC000D040CDBFDEBF5C018E010E5D1F4FC8010C
:105DD0000E9444166C01A2E4EA2EF12CEC0EFD1E8A
:105DE000D7014C91CE010196B80150E00E945A496A
:105DF000F701E080D7FE03C000E513E202C004E52E
:105E000013E2EE2029F04E010894811C911C04C07D
:105E1000F0E58F2EF6E29F2EFE01ED5BFF4F208115
:105E2000FE01EC5BFF4F3081FE01EB5BFF4F4081D9
:105E3000FE01EA5BFF4F5081FE01E95BFF4F60818D
:105E4000FE01E85BFF4F7081FE01EE0DF11D118236
:105E50008DB79EB746978DBF9EBFEDB7FEB7319603
:105E6000ADB7BEB71196AD92BC92129784E596E29B
:105E70008283938304831583C682D782808691862A
:105E8000228713863487158646871786508B118A9A
:105E9000628B138A748B158A0E94D81AEDB7FEB7ED
:105EA0007696EDBFFEBFC85BDF4FCDBFDEBFCF91A3
:105EB000DF911F910F91FF90EF90DF90CF90BF90F7
:105EC000AF909F908F900895AC01DC010D90002061
:105ED000E9F71197A81BB90BFB01A0A3CB01BA01ED
:105EE0004A2F50E00E945A4981E090E008950F93B4
:105EF0001F93DF93CF9300D000D0CDB7DEB78C01D6
:105F0000CE0101960E947D16AC0197FF03C020E5EB
:105F100033E202C024E533E28DB79EB744978DBFCC
:105F20009EBFEDB7FEB73196ADB7BEB711960D93D4
:105F30001C9312978FE796E28283938324833583A1
:105F4000468357838981808711868A818287138659
:105F50008B81848715868C81868717868D81808BBF
:105F6000118A8E81828B138A0E94D81A8DB79EB7B0
:105F700044968DBF9EBF2696CDBFDEBFCF91DF91E9
:105F80001F910F910895CF92DF92EF92FF920F939E
:105F90001F93DF93CF930F920F92CDB7DEB76C01B3
:105FA000FA0162307105E4F182819381BE016F5F75
:105FB0007F4F0E94E225892B99F189810E94180E5A
:105FC0008C0197FF05C080E5E82E83E2F82E04C01F
:105FD000B4E5EB2EB3E2FB2EC8010E94591F2DB78A
:105FE0003EB72A5030402DBF3EBFEDB7FEB73196C9
:105FF000ADB7BEB71196CD92DC92129727E533E28A
:1060000022833383E482F582068317838087918716
:106010000E94D81AEDB7FEB73A96EDBFFEBF14C086
:1060200000D00F92ADB7BEB71196CD92DC92129709
:1060300087EA96E213968D939C9314970E94D81A40
:106040000F900F900F900F900F900F90CF91DF91C6
:106050001F910F91FF90EF90DF90CF9008950F93D5
:106060001F93DF93CF930F92CDB7DEB78C01CE0194
:1060700001960E94380EBC0197FF03C040E553E231
:1060800002C044E553E28981882319F026EC36E208
:1060900002C029EC36E28DB79EB70A978DBF9EBF2E
:1060A000EDB7FEB73196ADB7BEB711960D931C9301
:1060B000129787E593E282839383448355836683B3
:1060C0007783208731870E94D81A8DB79EB70A96AA
:1060D0008DBF9EBF0F90CF91DF911F910F910895BB
:1060E000EF92FF920F931F93CF93DF937C01FA01FE
:1060F000623071050CF441C0C281D381CE0169ECDC
:1061000076E20E947549009711F480E008C0CE0144
:1061100066EC76E20E947549009779F581E00E946D
:10612000600EEC0197FF03C000E513E202C004E536
:1061300013E2CE010E94591F2DB73EB72A503040BE
:106140002DBF3EBFEDB7FEB73196ADB7BEB71196C6
:10615000ED92FC92129727E533E222833383048386
:106160001583C683D783808791870E94D81AEDB79D
:10617000FEB73A96EDBFFEBF14C000D00F92ADB788
:10618000BEB71196ED92FC9212978DEC96E21396A3
:106190008D939C9314970E94D81A0F900F900F9094
:1061A0000F90DF91CF911F910F91FF90EF90089585
:1061B000EF92FF920F931F93CF93DF937C010E9486
:1061C000E60FEC0197FF03C000E513E202C004E50F
:1061D00013E2CE010E94591F2DB73EB72A5030401E
:1061E0002DBF3EBFEDB7FEB73196ADB7BEB7119626
:1061F000ED92FC92129727E533E2228333830483E6
:106200001583C683D783808791870E94D81A2DB7BC
:106210003EB7265F3F4F2DBF3EBFDF91CF911F910D
:106220000F91FF90EF900895CF92DF92EF92FF923F
:106230000F931F93DF93CF93CDB7DEB7A397CDBF57
:10624000DEBF6C018A0133E0E32EF12CEC0EFD1E63
:1062500081E2D7011D928A95E9F764307105ECF06F
:10626000FA0182819381B7010E94642F892B09F47E
:106270006EC0D80116968D919C911797BE016F5FE5
:106280007F4F0E94E225892B09F461C0F8016481E7
:10629000758149815A81C7012BC06330710581F432
:1062A000DA0112968D919C911397B7010E94642F89
:1062B000892B09F44CC0F80164817581C70116C0AF
:1062C0006230710561F4DA0112968D919C911397F9
:1062D000B7010E94642F892BD1F1C70105C061303D
:1062E0007105A9F580E090E060E070E040E050E0EA
:1062F0000E941F178C0197FF05C020E5E22E23E2C4
:10630000F22E04C094E5E92E93E2F92EC8010E9412
:10631000591FEDB7FEB73A97EDBFFEBF3196ADB747
:10632000BEB71196CD92DC92129727E533E2228315
:106330003383E482F58206831783808791870E94E6
:10634000D81AEDB7FEB73A96EDBFFEBF14C000D025
:106350000F92ADB7BEB71196CD92DC9212978CEE2C
:1063600096E213968D939C9314970E94D81A0F90DF
:106370000F900F900F90A396CDBFDEBFCF91DF910E
:106380001F910F91FF90EF90DF90CF9008958F9223
:106390009F92AF92BF92CF92DF92EF92FF920F93B4
:1063A0001F93DF93CF9300D00F92CDB7DEB74C0190
:1063B0008A0119821A821B821C8263307105A4F043
:1063C000DA0112968D919C911397BE016F5F7F4FFA
:1063D0000E94E225892B09F475C0F801848195811A
:1063E000BE016D5F7F4F0CC06230710509F06AC05D
:1063F000DA0112968D919C911397BE016F5F7F4FCA
:106400000E94E225892B09F45DC069817A81882781
:1064100077FD8095982F4B810E94A7175C0100970C
:1064200059F588EE93E020E233E0F9013197F1F776
:106430000197D9F749815A81662757FD6095762FD4
:10644000CB80DC80809127309091283028E030E0AC
:1064500000E010E0E1E0EE2EF12C0E94E8219C012A
:1064600097FD45C088EE93E020E233E0F9013197D3
:10647000F1F70197D9F705C097FF03C000E513E2D4
:1064800002C004E513E2C5010E94591FEDB7FEB733
:106490003A97EDBFFEBF3196ADB7BEB711968D925C
:1064A0009C92129727E533E222833383048315837A
:1064B000A682B782808791870E94D81AEDB7FEB76F
:1064C0003A962BC000D00F92ADB7BEB711968D9201
:1064D0009C9212978FE097E213968D939C9314975A
:1064E0000E94D81A0F900F900F900F9018C000D0F4
:1064F00000D0EDB7FEB73196ADB7BEB711968D920D
:106500009C92129789E397E2828393832483358355
:106510000E94D81AEDB7FEB73696EDBFFEBF24969F
:10652000CDBFDEBFCF91DF911F910F91FF90EF9014
:10653000DF90CF90BF90AF909F908F900895EF9293
:10654000FF920F931F93CF93DF937C010E9404105F
:10655000EC0197FF03C000E513E202C004E513E27B
:10656000CE010E94591F2DB73EB72A5030402DBF93
:106570003EBFEDB7FEB73196ADB7BEB71196ED92FF
:10658000FC92129727E533E2228333830483158339
:10659000C683D783808791870E94D81A2DB73EB7CC
:1065A000265F3F4F2DBF3EBFDF91CF911F910F91CF
:1065B000FF90EF9008954F925F926F927F928F922B
:1065C0009F92AF92BF92CF92DF92EF92FF920F9382
:1065D0001F93CF93DF93582E492EEB013A014801C8
:1065E000590100D00F92EDB7FEB73196ADB7BEB7E7
:1065F00011968C9391838DE69AE2828393830E9415
:10660000D81A0F900F900F900F902097E1F0CE01C5
:106610000E94591FEDB7FEB73897EDBFFEBF319608
:10662000ADB7BEB711965C92418220E73AE2228371
:106630003383C483D583868397830E94D81AEDB7AA
:10664000FEB738965BC081149104A104B10409F42B
:1066500040C06301EE24D7FCE094FE2C2DB73EB77A
:10666000225130402DBF3EBF0DB71EB70F5F1F4FE9
:10667000ADB7BEB711965C92F801418283E89AE209
:106680008283938364827582D80116968D929D923F
:10669000AD92BC921997C701B601A50194010E9461
:1066A000A445F8012287338744875587C701B6017F
:1066B000A50194010E94A445D8011E966D937D9377
:1066C0008D939C9351970E94D81AEDB7FEB772969E
:1066D00015C000D000D0EDB7FEB73196ADB7BEB74C
:1066E00011965C92418289EB9AE282839383648261
:1066F00075820E94D81AEDB7FEB73696EDBFFEBF81
:10670000DF91CF911F910F91FF90EF90DF90CF908D
:10671000BF90AF909F908F907F906F905F904F90C1
:1067200008950F931F93CF93DF93182F092FEB0139
:1067300000D00F92EDB7FEB73196ADB7BEB7119648
:106740008C9391838FED9AE2828393830E94D81A6F
:106750000F900F900F900F901C161D06DCF4CE01C9
:1067600060E570E00E949145892BA1F400D00F9262
:10677000EDB7FEB73196ADB7BEB711961C93018346
:106780008DE69AE2828393830E94D81A0F900F902D
:106790000F900F90DF91CF911F910F910895AF92BD
:1067A000BF92CF92DF92EF92FF920F931F93CF93FE
:1067B000DF93EC01B62EA72E88899989892B71F079
:1067C0008C819D812E813F81AC01429FC001439FFE
:1067D000900D529F900D11246C0104C0CA88DB8873
:1067E000EC88FD886C857D85888599850E94692067
:1067F000EA8DFB8D309749F08C0120E030E08C8DE4
:106800009D8D6B2D7A2DA60119958A819B810E9401
:10681000AA46888199810E94CB1488899989892BFD
:1068200021F48E899F890E94CB14CE010E94AA4632
:106830008B2D9A2DDF91CF911F910F91FF90EF90AB
:10684000DF90CF90BF90AF9008958F929F92AF92BC
:10685000BF92CF92DF92EF92FF920F931F93CF934D
:10686000DF934C017B016A01590181E090E06EE108
:1068700070E00E94E145EC01009719F480E090E09F
:1068800010C0EC82FD82C88ED98EAA8EBB8E0C8F72
:106890001D8FC7010E94FD458A839B83009731F4B9
:1068A000CE016DEF7FEF0E94CF3323C080E090E0F8
:1068B00060E070E00E94E415BC018883998397FD35
:1068C00014C06DE87FE2A4010E94DA12BC0197FDBA
:1068D0000CC08881998161E070E046E854E39E0134
:1068E0000E949A12BC0197FF02C0CE01DCCF8881C2
:1068F0009981DF91CF911F910F91FF90EF90DF90E1
:10690000CF90BF90AF909F908F900895CF93DF93DB
:10691000EC01CB010E948515BC018E8B9F8B97FFEC
:1069200004C0CE010E94CF3314C063EF74E3AE0104
:106930000E944A0D8E899F896CEA74E3AE010E9421
:10694000650D0E940C20A0E0B0E088879987AA8797
:10695000BB87DF91CF910895CF93DF939B01EC012B
:1069600088899989892BE1F5452B61F40E940C20D7
:10697000A0E0B0E08C879D87AE87BF87CE0160E046
:1069800070E00BC06A817B814C815D81C9010E94EE
:106990006D11BC0197FF04C0CE010E94CF3320C00F
:1069A000EE81FF813196EE83FF839C01442737FD02
:1069B0004095542F8A899B89AC89BD89820F931F8A
:1069C000A41FB51F8A8B9B8BAC8BBD8B288D398DFB
:1069D0002115310529F08C8D9D8DBF01F901199587
:1069E000DF91CF9108952F923F924F925F926F92D5
:1069F0007F928F929F92AF92BF92CF92DF92EF924F
:106A0000FF920F931F93CF93DF93EC01452B19F463
:106A10006CEF7FEFB2C088899989892B89F50F9235
:106A20000F9281EE9AE2ADB7BEB711968D939C930B
:106A300012970E942F1EEDB7FEB73897EDBFFEBF2D
:106A400031968CEF9AE2ADB7BEB711968D939C93B9
:106A500012978FE09BE28283938382EB90E08483A2
:106A600095838CEB9FE28683978380E29BE280870D
:106A700091870E942F1EEDB7FEB73A96EDBFFEBF7D
:106A80000E940C20A0E0B0E088879987AA87BB8786
:106A9000EE24FF2451EE252E5AE2352E4CEF442EE3
:106AA0004AE2542E3FE0632E3BE2732E25E1822E14
:106AB00021E0922E94ECA92E9FE2B92E8BE2C82EF3
:106AC0008BE2D82E47C06A817B81600F711F401B0B
:106AD000510B888199810E942611BC0197FD31C01C
:106AE000080F191F4C815D810417150760F3041707
:106AF000150709F457C00F920F92ADB7BEB71196A4
:106B00002D923C9212970E942F1EEDB7FEB7389738
:106B1000EDBFFEBF3196ADB7BEB711964D925C92F8
:106B200012976282738284829582A682B782C0861F
:106B3000D1860E942F1EEDB7FEB73A96EDBFFEBF7D
:106B400031C0CE011AC08C8D9D8DB7011995089466
:106B5000E11CF11C8E819F81E816F90618F400E013
:106B600010E0C0CF0E940C20A0E0B0E08C879D8791
:106B7000AE87BF87CE0160E070E00E94CF33DF9127
:106B8000CF911F910F91FF90EF90DF90CF90BF902A
:106B9000AF909F908F907F906F905F904F903F90BD
:106BA0002F900895E88DF98D309769F6D0CF4F92E8
:106BB0005F926F927F928F929F92AF92BF92CF928D
:106BC000DF92EF92FF920F931F93CF93DF932C01ED
:106BD0003B014A0159014115510509F455C02115E0
:106BE000310509F451C06115710509F44DC081E00A
:106BF00090E06EE170E00E94E145EC01009719F42D
:106C00004DEF5FEF43C08E829F82AC82BD82088FC2
:106C1000198FEA8EFB8ECC8EDD8E81E090E0888B22
:106C2000998BC5010E94FD458A839B83009721F4BF
:106C3000CE016DEF7FEF13C080E090E060E070E088
:106C40000E94E415BC018883998397FD07C0B201B7
:106C5000A3010E944912BC0197FF05C0CE010E940A
:106C6000CF33AC0113C08881998163EF74E3AE0127
:106C70000E944A0D888199816CEA74E3AE010E94FA
:106C8000650D4881598102C04EEF5FEFCA01DF9167
:106C9000CF911F910F91FF90EF90DF90CF90BF9019
:106CA000AF909F908F907F906F905F904F900895DE
:106CB0002F923F924F925F926F927F928F929F920C
:106CC000AF92BF92CF92DF92EF92FF920F931F93FA
:106CD000DF93CF9300D000D0CDB7DEB75C013B018E
:106CE0006A0180918D2F90918E2FA0918F2FB0915E
:106CF000902F89839A83AB83BC8301E010E038E84E
:106D0000832E33E1932E20E034E02D833E83412C0B
:106D100024E0522E2224332470C0F801EE0FFF1F0E
:106D2000EC0DFD1DE080F180C7016FE37BE20E9466
:106D30007549009789F40F5F1F4F061517050CF072
:106D4000EEC0F801EE0FFF1FEC0DFD1D808191815B
:106D50000E940D494C014FC0C70162E47BE20E94D2
:106D60007549009791F40F5F1F4F061517050CF03A
:106D7000D6C0F801EE0FFF1FEC0DFD1D8081918143
:106D80000E940D498D839E8336C0C70165E47BE276
:106D90000E947549009789F40F5F1F4F061517056C
:106DA0000CF0BDC0F801EE0FFF1FEC0DFD1D808142
:106DB00091810E940D492C011EC0C70168E47BE24D
:106DC0000E947549009721F4F1E02F2E312C13C059
:106DD000C7016BE47BE20E947549009719F42224F5
:106DE000332409C0C701BE016F5F7F4F0E9408189E
:106DF000892B09F494C00F5F1F4F061517050CF47B
:106E00008CCF21143104C9F089819A81AB81BC8176
:106E10000097A105B10509F482C0CE010196B40125
:106E20004D815E81920101E913E3EBEDEE2EE2E389
:106E3000FE2E65010E94D73509C0C401B20141E9A7
:106E400053E32BED32E385010E9425348C0197FF3B
:106E50001BC00E94591FADB7BEB71A97ADBFBEBFCA
:106E6000EDB7FEB731961196AD92BC9212972EE413
:106E70003BE2228333832BE53BE224833583068385
:106E800017838087918743C0232859F1CE0101964B
:106E90000E9496192DB73EB72E5030402DBF3EBFF1
:106EA000EDB7FEB73196ADB7BEB71196AD92BC92B5
:106EB00012972FE53BE22283338384839583868276
:106EC00097822D813E8120873187428653860487B1
:106ED00015870E94D81A8DB79EB70E968DBF9EBF9C
:106EE00032C0ADB7BEB71A97ADBFBEBFEDB7FEB7E4
:106EF00031961196AD92BC92129780E99BE2828303
:106F000093838482958246825782008711870E94EC
:106F1000D81AEDB7FEB73A96EDBFFEBF14C000D049
:106F20000F92ADB7BEB71196AD92BC9212978BEB94
:106F30009BE213968D939C9314970E94D81A0F90FE
:106F40000F900F900F902696CDBFDEBFCF91DF91AF
:106F50001F910F91FF90EF90DF90CF90BF90AF9077
:106F60009F908F907F906F905F904F903F902F9069
:106F700008952F923F924F925F926F927F928F92DD
:106F80009F92AF92BF92CF92DF92EF92FF920F93B8
:106F90001F93DF93CF93CDB7DEB7EE97CDBFDEBFA4
:106FA0009C016DAF7EAFDE011196ECECFFE284E355
:106FB00001900D928150E1F7D901ED90FD900D9176
:106FC0001C91C801B70120E831E541E050E00E9482
:106FD000A445C901DA015C016D01C801B70120E8CF
:106FE00031E541E050E00E94A445AC01CB01DA015B
:106FF0007C018D010DC080E891E5A1E0B0E0E80ED4
:10700000F91E0A1F1B1F0894A108B108C108D10866
:1070100017FDF1CF0DC080E89EEAAEEFBFEFE80E9E
:10702000F91E0A1F1B1F0894A11CB11CC11CD11CF6
:1070300090E8E91691E5F90691E0090790E0190753
:1070400050F7C801B70120E13EE040E050E00E9467
:10705000C645ADADBEAD12962C93C801B70120E177
:107060003EE040E050E00E94C645162F072FF82E64
:10707000E92E2CE330E040E050E00E94C645EDAD43
:10708000FEAD2183612F702F8F2D9E2D2CE330E0DC
:1070900040E050E00E94C645ADADBEAD6C93C60168
:1070A000B5016C5F7F4F8F4F9F4F27E030E040E08E
:1070B00050E00E94C645EDADFEAD6187E2EB2E2E9D
:1070C000E7E03E2E412C512C2EC1C601B5012DE624
:1070D00031E040E050E00E94C64539014A01EE240B
:1070E000FF248701C601B5012DE631E040E050E004
:1070F0000E94C64597FF05C071E0E72EF12C012DD7
:10710000112DD401C3018E199F09A00BB10B820D63
:10711000931DA41DB51D8DAB9EABAFABB8AF4201A7
:107120003101089461087108810891080197A1094B
:10713000B10989AF9AAFABAFBCAFC401B30124E0D2
:1071400030E040E050E00E94C64579018A01C40168
:10715000B3012CE93FEF4FEF5FEF0E94C645E20E0F
:10716000F31E041F151FEA0CFB1C0C1D1D1DC40182
:10717000B30120E931E040E050E00E94C645E20E54
:10718000F31E041F151FAA24BB246501C401B3010B
:1071900024E630E040E050E00E94C64597FF05C07D
:1071A00061E0A62EB12CC12CD12CAE0CBF1CC01E90
:1071B000D11EEE24FF248701C401B30124E030E096
:1071C00040E050E00E94C64597FF05C051E0E52E23
:1071D000F12C012D112DAE18BF08C00AD10AEE24E2
:1071E000FF248701C401B30120E931E040E050E011
:1071F0000E94C64597FF05C041E0E42EF12C012D09
:10720000112DD601C5018E199F09A00BB10B7C0170
:107210008D0169AD7AAD8BAD9CAD20E73EEF4FEFB0
:107220005FEF0E94C645E20EF31E041F151F69ADF5
:107230007AAD8BAD9CAD24E630E040E050E00E949A
:10724000C645E20EF31E041F151F69AD7AAD8BAD66
:107250009CAD24E030E040E050E00E94C645E21AD8
:10726000F30A040B150B8DA99EA9AFA9B8AD281A76
:10727000390A4A0A5B0AC201B1012DE631E040E059
:1072800050E00E945245E60EF71E081F191FAA245F
:10729000BB24650169AD7AAD8BAD9CAD20E931E0D1
:1072A00040E050E00E94C64597FF05C031E0A32EA4
:1072B000B12CC12CD12CAE0CBF1CC01ED11EEE2493
:1072C000FF24870169AD7AAD8BAD9CAD24E030E041
:1072D00040E050E00E94C64597FF05C021E0E22E45
:1072E000F12C012D112DAE0CBF1CC01ED11EEE24A1
:1072F000FF24870169AD7AAD8BAD9CAD24E630E00B
:1073000040E050E00E94C64597FF05C091E0E92E9D
:10731000F12C012D112DAE18BF08C00AD10A2DA8DD
:107320003EA84FA858ACD7FCD0CE83E0E82EF12C75
:10733000012D112DE220F32004211521E114F10487
:1073400001051105F9F4C201B10124E630E040E085
:1073500050E00E94C645611571058105910569F4EB
:10736000C201B10120E931E040E050E00E94C64591
:10737000611571058105910529F48EE691E0A0E083
:10738000B0E004C08DE691E0A0E0B0E0A816B90638
:10739000CA06DB060CF099CEC1018C569740ADAD04
:1073A000BEAD15968D939C9316971796AD92BC9291
:1073B0001897E114F1040105110519F020E030E0FF
:1073C00022C0C201B10124E630E040E050E00E945A
:1073D000C645611571058105910519F021E030E080
:1073E00012C000E010E0C201B10120E931E040E04C
:1073F00050E00E94C645611571058105910511F4A3
:1074000001E010E098018AE190E0FC012E9FC001AC
:107410002F9F900D3E9F900D1124FE013196E80F95
:10742000F91F2BE030E040E050E004C02150304034
:1074300040405040868997893297A0E0B0E0A81676
:10744000B906CA06DB0694F3EDADFEAD2483A81A97
:10745000B90ACA0ADB0A8A2D8F5F838381E090E034
:10746000EE96CDBFDEBFCF91DF911F910F91FF90C0
:10747000EF90DF90CF90BF90AF909F908F907F90D4
:107480006F905F904F903F902F9008950F931F93B0
:10749000CF93DF93182F092FDB01EA0161157105E6
:1074A00009F5CA010E94591F2DB73EB72850304038
:1074B0002DBF3EBFEDB7FEB73196ADB7BEB7119643
:1074C0001C9301832CEE3BE22283338384839583D8
:1074D000C683D7830E94D81ACDB7DEB72896CDBF12
:1074E000DEBF3AC02DB73EB7205130402DBF3EBF62
:1074F000EDB7FEB73196CDB7DEB7898391838CE0C7
:107500009CE28283938315968D919C911697845962
:10751000984F8483958314968C91149790E00196EC
:107520008683978313968C91139780871186129682
:107530008C9112978287138611968C91119784876C
:1075400015868C91868717860E94D81A2DB73EB76C
:10755000205F3F4F2DBF3EBFDF91CF911F910F9115
:107560000895CF93DF93EC018C819D811816190645
:1075700014F40E94CB148E819F81009711F00E9419
:107580000121CE010E94AA46DF91CF9108956F920A
:107590007F928F929F92AF92BF92CF92DF92EF92A3
:1075A000FF920F931F93DF93CF93CDB7DEB7E09792
:1075B000CDBFDEBF4C018B015A013E010894611C16
:1075C000711C80E3F30111928A95E9F783E28983C4
:1075D00081E090E068E070E00E94E1457C01009766
:1075E00019F40DEF1FEF3FC081E090E060E070E024
:1075F0000E94E4156C011816190684F5F701008342
:107600001183A282B3828483958388E893E160E04A
:1076100070E048EB5BE397010E947321F7018683DA
:107620009783892BD9F0C601B4014BE750E00E9443
:1076300049128C010097A1F4C6016CEC7BE3A70111
:107640000E94650D97FD08C0C601B30140E350E0FC
:107650000E94261197FF07C08C0102C00DEF1FEF9B
:10766000C7010E94B13AC801E096CDBFDEBFCF91FD
:10767000DF911F910F91FF90EF90DF90CF90BF901F
:10768000AF909F908F907F906F900895CF92DF92F0
:10769000EF92FF920F931F93DF93CF9300D00F923F
:1076A000CDB7DEB77C01FA01623071050CF440C041
:1076B000828193818E010F5F1F4FB8010E940818CD
:1076C000892BB1F1C80166E47AE3A7010E94C73AA9
:1076D0008C0197FF05C0A6E3CA2EACE2DA2E04C0E7
:1076E000FAE3CF2EFCE2DF2EC8010E94591F2DB70E
:1076F0003EB72A5030402DBF3EBFEDB7FEB73196A2
:10770000ADB7BEB71196ED92FC9212972DE33CE215
:1077100022833383C482D58206831783808791872F
:107720000E94D81AEDB7FEB73A96EDBFFEBF14C05F
:1077300000D00F92ADB7BEB71196ED92FC921297A2
:107740008AE49CE213968D939C9314970E94D81A16
:107750000F900F900F900F902496CDBFDEBFCF916A
:10776000DF911F910F91FF90EF90DF90CF900895E0
:10777000CF93DF93EB01E881F981309739F08A816B
:107780009B8160E070E04FEE5FEF1995CE010E94A3
:10779000B13ADF91CF910895AF92BF92CF92DF922D
:1077A000EF92FF920F931F93DF93CF93CDB7DEB786
:1077B0002E97CDBFDEBF6B017A018C01403351059E
:1077C00038F4AA24BB2480EFC82E8FEFD82E2EC009
:1077D000CA010E94FD455C01009729F4BDEFCB2E44
:1077E000BFEFDB2E23C0C601B501A7010E946D11BA
:1077F0006C018E159F05D1F4D50190966D917D9108
:107800008D919C9193970E94051860587E478A4AF3
:10781000934869837A838B839C83F894CE01019685
:10782000BE016B5F7F4F0E94B9377894D801ED910C
:10783000FC911197309749F012968D919C91139776
:10784000BE016B5F7F4FA6011995C5010E94AA4634
:10785000C8010E94B13A2E96CDBFDEBFCF91DF9115
:107860001F910F91FF90EF90DF90CF90BF90AF905E
:107870000895CF92DF92EF92FF920F931F93D82E2D
:10788000C92ECB018A0179010E94961900D000D03F
:10789000EDB7FEB73196ADB7BEB71196DC92C18297
:1078A00021E83CE222833383848395830E94D81AA3
:1078B0000F920F92EDB7FEB73196ADB7BEB71196E6
:1078C000DC92C1828EE99CE28283938304831583D8
:1078D000E682F7820E94D81A8DB79EB708968DBFB0
:1078E0009EBF1F910F91FF90EF90DF90CF90089572
:1078F000CF92DF92EF92FF920F931F93CF93DF937C
:10790000D82EC92EEB01790101151105A1F4CA0188
:107910000E9496192DB73EB72A5030402DBF3EBF6A
:10792000EDB7FEB73196ADB7BEB71196DC92C18206
:1079300024EC3CE213C003301105F9F4CA010E94A3
:107940009619ADB7BEB71A97ADBFBEBFEDB7FEB7BC
:1079500031961196DC92C18224EE3CE2228333837D
:10796000C483D58386839783E086F1860E94D81AE4
:107970002DB73EB7265F3F4F20C0CA010E9496191F
:10798000ADB7BEB71C97ADBFBEBFEDB7FEB7319662
:107990001196DC92C18221E23DE222833383C483CB
:1079A000D58386839783E086F186028713870E94BA
:1079B000D81A2DB73EB7245F3F4F2DBF3EBFDF9192
:1079C000CF911F910F91FF90EF90DF90CF9008958E
:1079D000CF93DF93EC01888D998D1816190614F456
:1079E0000E94CB148A8D9B8D009711F00E9401217B
:1079F0008C819D810E94AA46CE010E94AA46DF91F9
:107A0000CF9108954F925F926F927F928F929F9243
:107A1000AF92BF92CF92DF92EF92FF920F931F939C
:107A2000CF93DF935C014B01D42EC52E3901280181
:107A300081E090E06CE170E00E94E145EC0100978C
:107A400009F445C00D2D1C2DB801685F7F4F81E002
:107A500090E00E94E1458C839D830097A9F182E02C
:107A600090E061E070E00E94E415888F998F18160D
:107A7000190654F565E07FE3AE010E94650DF5013E
:107A800080819181A281B38188839983AA83BB83FA
:107A90008A8A9B8A0E831F831E861F866886798644
:107AA0004A865B86EC86FD8680E090E060E070E0D0
:107AB0004EE55EE39E010E9473218A8F9B8F892B86
:107AC00019F020E030E005C0CE010E94E83C2DEF27
:107AD0003FEFC901DF91CF911F910F91FF90EF9080
:107AE000DF90CF90BF90AF909F908F907F906F90DE
:107AF0005F904F9008952F923F924F925F926F92B6
:107B00007F928F929F92AF92BF92CF92DF92EF922D
:107B1000FF920F931F93DF93CF9300D00F92CDB7B7
:107B2000DEB74C015B016A0180918D2F90918E2F01
:107B3000A0918F2FB091902F89839A83AB83BC83C0
:107B400001E010E063E0462E512C50E2652E712CCE
:107B50001E010894211C311C40C0F801EE0FFF1FCC
:107B6000EC0DFD1DE080F180C70169E47DE20E941B
:107B70007549009789F40F5F1F4F0A151B050CF01C
:107B800073C0F801EE0FFF1FEC0DFD1D8081918188
:107B90000E940D492C011FC0C7016CE47DE20E94C8
:107BA0007549009789F40F5F1F4F0A151B050CF0EC
:107BB0005BC0F801EE0FFF1FEC0DFD1D8081918170
:107BC0000E940D493C0107C0C701B1010E9408187D
:107BD000892B09F449C00F5F1F4F0A151B050CF4D0
:107BE000BCCF89819A81AB81BC810097A105B10589
:107BF000D9F1CE010196B201A30128E73CE309E3E4
:107C00001CE374010E94023D8C0197FF05C09FE4B4
:107C1000E92E9DE2F92E04C083E5E82E8DE2F82ED0
:107C2000C8010E94591F2DB73EB72A5030402DBFC2
:107C30003EBFEDB7FEB73196ADB7BEB711968D9288
:107C40009C92129726E53DE222833383E482F582FB
:107C500006831783808791870E94D81AEDB7FEB7F5
:107C60003A96EDBFFEBF14C000D00F92ADB7BEB7BD
:107C700011968D929C92129783E69DE213968D93B6
:107C80009C9314970E94D81A0F900F900F900F900A
:107C90002496CDBFDEBFCF91DF911F910F91FF9052
:107CA000EF90DF90CF90BF90AF909F908F907F909C
:107CB0006F905F904F903F902F900895CF92DF92FA
:107CC000EF92FF920F931F93CF93DF93EB010C8101
:107CD0001D81288939898A899B892817390779F470
:107CE000EA85FB85309739F04C895D892E893F897B
:107CF0008C859D851995CE010E94E83C7DC0CE8083
:107D0000DF8088E090E0C80ED91E88E0F80180830B
:107D10001182128213828E859F850E94D017F801EE
:107D200084839583888999890E94D017F801868376
:107D30009783760120E030E040E050E011C0708190
:107D400060E0818190E0862B972B3296A0E0B0E036
:107D5000280F391F4A1F5B1F8EEF9FEFE80EF91E99
:107D600092E0E916F10458F7C6018E7FF801E80F9A
:107D7000F91FC816D90641F0908180E0A0E0B0E07C
:107D8000280F391F4A1F5B1FCA01AA27BB27407053
:107D90005070280F391F4A1F5B1F40FF09C0CA01DE
:107DA000AA27BB2740705070280F391F4A1F5B1F3E
:107DB000C9010E94D01780959095F8018283938322
:107DC000888D998DB801A6019E0100E010E00E9407
:107DD000C8108C159D0529F48C899D8901968C8B82
:107DE0009D8B8A8D9B8D68EE73E00E94E31F8889CE
:107DF00099890196888B998BDF91CF911F910F9173
:107E0000FF90EF90DF90CF9008958F929F92AF9266
:107E1000BF92CF92DF92EF92FF920F931F93CF9377
:107E2000DF93E82E992E8B01EA01CA010E94FD45DD
:107E30006C010097C1F1C801B601AE010E946D113D
:107E40005C018C179D0779F58CE1A816B10458F1F7
:107E5000CE2DD92D86010C5E1F4FF80184819581AE
:107E60000E94D4172E853F8582179307E1F48E89EF
:107E70009F8901968E8B9F8B8884998481149104AD
:107E800091F0EC84FD84F801868197810E94D417DB
:107E90009C01A601445F5F4FF8010081C701B50155
:107EA00010E0F4011995C6010E94AA46DF91CF9116
:107EB0001F910F91FF90EF90DF90CF90BF90AF9008
:107EC0009F908F9008952F923F924F925F926F9262
:107ED0007F928F929F92AF92BF92CF92DF92EF925A
:107EE000FF920F931F93DF93CF9300D00F92CDB7E4
:107EF000DEB75C013B0129833A83280161157105D6
:107F000019F48B839C830BC0FB010190F081E02D61
:107F1000E80FF91FEB83FC83FB01108211828A01B9
:107F20008824992415010894211C311C50C0EB8130
:107F3000FC819081992309F452C0F8018081C92EF7
:107F4000DD24C7FCD0944114510431F0E82EFF2405
:107F5000E7FCF094C60109C0992787FD90950E941F
:107F60003B497C01C6010E943B49E816F90629F10C
:107F7000F8018081F501F0804114510449F0C82EC8
:107F8000DD24C7FCD0948F2D992787FD90950CC0D8
:107F9000992787FD90950E943B496C018F2D992769
:107FA00087FD90950E943B49C816D90619F0AB820F
:107FB000BC8208C02B823C8205C08B819C810196CB
:107FC0008B839C830F5F1F4F0894811C911CE98158
:107FD000FA818E169F0608F4AACF00E010E0611423
:107FE000710439F08B819C818A199B09F30180838C
:107FF0009183C8012496CDBFDEBFCF91DF911F9141
:108000000F91FF90EF90DF90CF90BF90AF909F9037
:108010008F907F906F905F904F903F902F9008953A
:10802000CF92DF92EF92FF920F931F93CF93DF9344
:108030006C017B01DB010D900020E9F78D010150FF
:108040001040061B170BC0E0D0E00EC0B7016C0F4C
:108050007D1FA8014C1B5D0BC6010E9426119C01CF
:1080600097FD07C0C80FD91FC017D1077CF320E0C8
:1080700030E0C901DF91CF911F910F91FF90EF90F8
:10808000DF90CF9008958F929F92AF92BF92CF9240
:10809000DF92EF92FF920F931F93CF93DF934C01E8
:1080A0005B016A0180E490E00E94FD45F82EE92E14
:1080B00000E010E020C0E601C01BD10BC134D105A7
:1080C00014F0C0E4D0E0B501600F711F8F2D9E2D1C
:1080D000AE010E944349C4016F2D7E2DAE010E9466
:1080E0002611EC0197FF05C08F2D9E2D0E94AA46F8
:1080F0000BC0080F191F0C151D05ECF28F2D9E2DBE
:108100000E94AA46C0E0D0E0CE01DF91CF911F913E
:108110000F91FF90EF90DF90CF90BF90AF909F9026
:108120008F900895EF92FF920F931F937C018B0124
:10813000CB010E944C49AC01C701B8010E944340E9
:108140001F910F91FF90EF900895EF92FF920F9380
:108150001F93DF93CF93CDB7DEB7AC97CDBFDEBF14
:108160007C01009719F42FEF3FEFE2C08EE49FE20D
:10817000A1E4B0E08B8F9C8FAD8FBE8FFE017F9608
:108180008EE0DF011D928A95E9F7C70167E876E086
:108190000E9492409C0197FDCBC08E010F5F1F4F44
:1081A000C80160E070E040E050E020E030E00E9474
:1081B000320F892B19F004E91DE204C0C8010E94A6
:1081C00096198C01C70162E776E00E9492409C01FB
:1081D00097FDAEC0C701B8010E9410409C0197FDF9
:1081E000A7C0C70167E576E00E9492409C0197FD19
:1081F0009FC0CE0105960E947D16892B99F52DB75B
:108200003EB7225130402DBF3EBFEDB7FEB731968D
:10821000CE014B96ADB7BEB711968D939C93129736
:1082200082E190E08283938388E99DE28483958351
:108230008D81868317828E81808711868F818287C8
:1082400013868885848715868985868717868A851B
:10825000808B118A0E94D1492DB73EB72E5E3F4FC9
:108260002DBF3EBFC70161E476E00E9492409C01B1
:1082700097FD5EC0C701BE01655E7F4F0E94104042
:108280009C0197FD55C0C70166E276E00E949240CE
:108290009C0197FD4DC0C70160E176E00E949240CD
:1082A0009C0197FD45C00E948D23ADB7BEB71897BE
:1082B000ADBFBEBFEDB7FEB731968E01055F1F4F54
:1082C00011960D931C93129720E130E022833383A3
:1082D00026EB3DE224833583868397830E94D14930
:1082E0002DB73EB7285F3F4F2DBF3EBFC701B80136
:1082F0000E9410409C0197FD1BC0C70165EF75E00F
:108300000E9492409C0197FD13C0C70168EC73E086
:108310000E9492409C0197FD0BC0C70160E272E091
:108320000E9492409C011816190614F420E030E0D7
:10833000C901AC96CDBFDEBFCF91DF911F910F91E8
:10834000FF90EF900895EF92FF920F931F93DF93AA
:10835000CF930F920F92CDB7DEB78C017B016BEB01
:108360007DE20E947549009799F1C8016DEB7DE2AD
:108370000E947549009761F1C80160EC7DE24CE014
:1083800050E00E948549009741F500D000D0EDB73C
:10839000FEB73196045F1F4FADB7BEB711960D9370
:1083A0001C9312978DEC9DE282839383CE010196FC
:1083B000848395830E94094A2DB73EB72A5F3F4FB9
:1083C0002DBF3EBF892B21F089819A810E946923AC
:1083D000C7010E94A5409C012FC0C8016AED7DE243
:1083E0000E9475490097A1F3C80166EE7DE20E94E4
:1083F0007549009781F4C7016FEC7DE00E949240BF
:108400009C0197FD19C0C7016AEE78E045EE54E083
:108410000E9443400BC0E114F10419F42FEF3FEF29
:108420000BC0C7016BE07EE00E9492409C011816D1
:10843000190614F420E030E0C9010F900F90CF919D
:10844000DF911F910F91FF90EF900895CF93DF93ED
:10845000EC018A819B81009721F00E94CB141A8243
:108460001B82DF91CF910895CF93DF93EC010E949F
:10847000264288819981009711F00E94CB14CE0189
:108480000E94AA46DF91CF910895EF92FF920F9339
:108490001F93CF93DF937C0181E090E066E870E06A
:1084A0000E94E145EC018C01009739F180E090E0F9
:1084B00060E070E00E94E4158883998397FD12C004
:1084C0006DE87FE2A7010E94DA12892B59F48881B6
:1084D000998161E070E045E852E49E010E949A12A1
:1084E000892B59F088819981009711F00E94CB1453
:1084F000CE010E94AA4600E010E0C801DF91CF91B2
:108500001F910F91FF90EF9008950F931F93CF93BA
:10851000DF93EC018A819B81892B19F0CE010E94A7
:108520002642888199810E9485158C0197FD0DC096
:108530006BE073E4AE010E944A0DC8016AEA72E47E
:10854000AE010E94650D0A831B83DF91CF911F91BD
:108550000F910895EF92FF920F931F93CF93DF93A4
:108560007C014115510509F44CC01FB7F894EC018A
:1085700026964138510514F040E850E0CB01BE0189
:108580000E946D119C011FBF97FD3EC0F7018281C3
:108590009381892BC9F180EF9DE260E070E0AE012C
:1085A00001E010E00E94633FFC01009769F1108236
:1085B000CE0163EF7DE244E050E00E9485490097E0
:1085C00001F5E7012A9601C021968881992787FD48
:1085D00090950E943349892BB9F71C2F0D2F01C0AC
:1085E00021968881992787FD90950E943349892B90
:1085F000B9F31882F70162817381812F902F0E9455
:10860000A341C7010E942642DF91CF911F910F9194
:10861000FF90EF900895DF93CF9300D00F92CDB7E6
:10862000DEB7452B39F0CB01BE016F5F7F4F0E9453
:10863000941002C00E9426422496CDBFDEBFCF9187
:10864000DF910895682F772767FD709580EA98E09D
:108650000E9471220895BF92CF92DF92EF92FF9213
:108660000F931F93DF93CF93CDB7DEB7A997CDBFFD
:10867000DEBF0E9477238FE090E06FE475E40E94F4
:108680004C230E94C4238FE090E00E94C82197FDF4
:108690006EC1B090A80680EA98E040E855E260E03C
:1086A00070E028E030E000E010E0E1E0EE2EF12C98
:1086B000CC24DD240E94E82197FD59C180EA99E08D
:1086C00040E051EE60E070E028E030E00E94E821F8
:1086D00097FD4DC180E090E061E772E240EA58E02A
:1086E00024E030E00E94621B7C01009709F43FC146
:1086F00080ED97E020E233E0F9013197F1F701973F
:10870000D9F788E892E26DE972E240EA59E00E9406
:10871000AD1697FD2CC180EA99E0809327309093A5
:10872000283088EE93E020E233E0F9013197F1F749
:108730000197D9F786EC94E4B7010E94380D8FEDCC
:1087400094E4B7010E94410DC70169E87EE240E070
:1087500050E00E94FE19C70163E97EE240E050E06C
:108760000E94FE19C7016BEB7EE240E050E00E94E0
:10877000FE19C70165EC7EE240E050E00E94FE1960
:10878000C7016FEC7EE240E050E00E94FE19C70195
:1087900069ED7EE240E050E00E94FE19C70163EE01
:1087A0007EE240E050E00E94FE19C7016DEE7EE2DD
:1087B00040E050E00E94FE19C70167EF7EE240E012
:1087C00050E00E94FE19C70161E57FE240E050E001
:1087D0000E94FE19C70161E07FE240E050E00E9484
:1087E000FE19C7016BE07FE240E050E00E94FE19F5
:1087F000C70165E17FE240E050E00E94FE19C70139
:108800006FE17FE240E050E00E94FE19C70169E29B
:108810007FE240E050E00E94FE19C70163E37FE27F
:1088200040E050E00E94FE19C7016DE37FE240E0A6
:1088300050E00E94FE19C70167E47FE240E050E08B
:108840000E94FE19C70165E67FE240E050E00E9409
:10885000FE19C7016BE57FE240E050E00E94FE197F
:10886000C7016DE97EE240E050E00E94FE19C701B9
:1088700067EA7EE240E050E00E94FE19C70161EB2A
:108880007EE240E050E00E94FE19C70165E77EE20B
:1088900040E050E00E94FE19C7016FE77EE240E031
:1088A00050E00E94FE19C7016FE67FE240E050E011
:1088B0000E94FE19C70169E77FE240E050E00E9494
:1088C000FE19C70163E87FE240E050E00E94FE1914
:1088D000C7016BE67EE240E050E00E94FE198FEF98
:1088E000B81681F566E172E088EA90EC0E94D8172C
:1088F00069837A838B839C8360E07FEF8FEF9FEFA8
:108900000E94D8176D837E838F8398878E01075FBF
:108910001F4FC80168EF7DE20E947E498AE089A767
:10892000C80163E07EE240E050E00E941F17CE01E4
:108930000196BE016B5F7F4F40E050E020E030E0E9
:108940000E94DD0F80EA98E00E94D422892B51F02A
:1089500080EA98E060E070E00E943023682FC70151
:108960000E94BB1C0E9416130E947720EBCF8FEF52
:108970009FEFA996CDBFDEBFCF91DF911F910F91E1
:10898000FF90EF90DF90CF90BF90089500D000D07F
:10899000EDB7FEB73196ADB7BEB711968D939C93E8
:1089A000129781E19EE282839383648375830E94A0
:1089B000D81A8DB79EB706968DBF9EBF08950F93A8
:1089C0001F93182F092F6115710571F500D00F92B3
:1089D000EDB7FEB73196ADB7BEB711968C939183C4
:1089E00083E29EE2828393830E94D81A809125308D
:1089F000909126300F900F900F900F90009709F4F0
:108A00004BC00E943442109225301092263000D084
:108A10000F92EDB7FEB73196ADB7BEB711961C9366
:108A2000018385E39EE230C0CB010E94961900D0FD
:108A300000D0EDB7FEB73196ADB7BEB711961C9317
:108A4000018325E43EE222833383848395830E945D
:108A5000D81A8DB79EB706968DBF9EBF80E590E071
:108A60000E9445428093253090932630892BA1F0B7
:108A700000D00F92EDB7FEB73196ADB7BEB71196E5
:108A80001C93018385E59EE2828393830E94D81A1A
:108A90000F900F900F900F901F910F9108950E94CB
:108AA00022200895629FD001739FF001829FE00D04
:108AB000F11D649FE00DF11D929FF00D839FF00D5D
:108AC000749FF00D659FF00D9927729FB00DE11D09
:108AD000F91F639FB00DE11DF91FBD01CF011124E6
:108AE0000895991B79E004C0991F961708F0961B0A
:108AF000881F7A95C9F780950895AA1BBB1B51E181
:108B000007C0AA1FBB1FA617B70710F0A61BB70BFD
:108B1000881F991F5A95A9F780959095BC01CD01A2
:108B2000089597FB092E07260AD077FD04D0E5DFCC
:108B300006D000201AF4709561957F4F0895F6F7DE
:108B4000909581959F4F0895A1E21A2EAA1BBB1BF9
:108B5000FD010DC0AA1FBB1FEE1FFF1FA217B30709
:108B6000E407F50720F0A21BB30BE40BF50B661F1F
:108B7000771F881F991F1A9469F7609570958095E3
:108B800090959B01AC01BD01CF01089597FB092E83
:108B900005260ED057FD04D0D7DF0AD0001C38F4CC
:108BA00050954095309521953F4F4F4F5F4F089519
:108BB000F6F790958095709561957F4F8F4F9F4FF9
:108BC00008950F931F93CF93DF93689F8001699F50
:108BD000100D789F100D1124C8010E94FD45EC0175
:108BE000009729F060E070E0A8010E946349CE017F
:108BF000DF91CF911F910F910895CF93DF93BC0127
:108C00008230910510F462E070E0A0914630B0919E
:108C10004730ED0140E050E0E0E0F0E021C0888125
:108C200099818617970769F48A819B81309719F09B
:108C30008283938304C08093463090934730FE0133
:108C400034C06817790738F44115510519F08417B5
:108C5000950708F4AC01FE018A819B819C01E90122
:108C60002097E9F641155105A9F1CA01861B970B1A
:108C7000049708F4BA01E0E0F0E02AC08D919C91DD
:108C8000119784179507F9F46417750781F4129604
:108C90008D919C911397309719F08283938304C030
:108CA0008093463090934730FD0132964FC0CA0101
:108CB000861B970BFD01E80FF91F619371930297D3
:108CC0008D939C9343C0FD01828193819C01D901C6
:108CD0001097A1F68091443090914530892B41F452
:108CE0008091672E9091682E809344309093453008
:108CF0004091692E50916A2E4115510541F44DB7AE
:108D00005EB78091652E9091662E481B590B20917D
:108D100044303091453024173507B0F4CA01821B26
:108D2000930B8617970780F0AB014E5F5F4F841758
:108D3000950750F0420F531F4093443050934530F5
:108D4000F9016193719302C0E0E0F0E0CF01DF919F
:108D5000CF910895CF93DF93009709F450C0EC01B1
:108D600022971A821B82A0914630B091473010970B
:108D700009F140E050E0AC17BD0708F1AA83BB83BE
:108D8000FE0121913191E20FF31FAE17BF0779F475
:108D90008D919C911197280F391F2E5F3F4F28838B
:108DA000398312968D919C9113978A839B834115E9
:108DB000510571F4C0934630D093473020C01296CD
:108DC0008D919C911397AD01009711F0DC01D3CFE9
:108DD000FA01C283D38321913191E20FF31FCE17A1
:108DE000DF0769F488819981280F391F2E5F3F4F73
:108DF000FA01208331838A819B8182839383DF916F
:108E0000CF9108958F929F92AF92BF92CF92DF92AF
:108E1000EF92FF920F931F93CF93DF938C010097F4
:108E200029F4CB010E94FD458C01BAC09EEFE92ECA
:108E30009FEFF92EE00EF11E5801A60EB71EAE14DC
:108E4000BF0408F4ABC08EEF882E8FEF982E8A0CEB
:108E50009B1CE7014881598146175707B8F04530F8
:108E6000510508F49DC0CA0104978617970708F4B6
:108E700097C042505040461B570BF401408351832A
:108E800068837983C5010E94AA468AC06B01C41A0F
:108E9000D50AE0914630F0914730C0E0D0E0A0E044
:108EA000B0E042C0E815F905A1F5208131812C150B
:108EB0003D0578F1C90102968C159D05A8F04E5F1D
:108EC0005F4F420F531FE70148835983228133814B
:108ED000109729F012962D933C93139761C020931D
:108EE0004630309347305CC0225030402C193D0949
:108EF00020833183109729F01296ED93FC931397FA
:108F000004C0E0934630F0934730F70160837183EB
:108F100047C080819181C817D90708F4EC01DF01AF
:108F2000828193819C01F901309709F0BBCF400FFA
:108F3000511F809144309091453084179507E9F492
:108F4000C617D707D0F42091692E30916A2E2115CB
:108F5000310541F42DB73EB78091652E9091662E74
:108F6000281B390BA216B306C8F4A0924430B09265
:108F70004530E7016883798313C0CB010E94FD452A
:108F8000EC01009759F0F70140815181B8010E942E
:108F90005A49C8010E94AA468E0102C000E010E0B2
:108FA000C801DF91CF911F910F91FF90EF90DF905B
:108FB000CF90BF90AF909F908F9008952F923F9247
:108FC0005F926F927F928F929F92AF92BF92CF9259
:108FD000DF92EF92FF920F931F93CF93DF938C0159
:108FE0001B01EA016115710519F0FB018083918372
:108FF000209749F0CE010297839728F020E030E0D7
:1090000040E050E0F6C0F801A1908F018A2D90E079
:109010000E943349892BB9F7FDE2AF1631F4F8010C
:10902000A1908F015524539407C0FBE2AF1619F4A9
:10903000F801A1908F015524209719F0C031D10576
:10904000C1F4F0E3AF1679F4F8018081883711F0AC
:10905000883549F4F801A1800E5F1F4FF2E05F2AC6
:10906000C0E1D0E006C0209721F480E3A816E9F41F
:1090700027C0C830D10531F1C930D10524F4C23040
:10908000D10531F50CC0CA30D10589F0C031D10508
:10909000F9F4C12CD12CE12CB8E0FB2E28C0C12C56
:1090A000D12CE12CA0E4FA2E22C0CAE0D0E0FCECE6
:1090B000CF2EFCECDF2EFCECEF2EFCE0FF2E17C0D9
:1090C000C8E0D0E0C12CD12CE12CE0E1FE2E0FC095
:1090D0009E01442737FD4095542F60E070E080E00A
:1090E00090E80E94A445C901DA016C017D0120E0ED
:1090F00030E040E050E060E03E01882477FC80945E
:10910000982C70EDB72EBA0CE9E0EB1570F48A2DAF
:1091100081548A3118F499ECB92E06C08A2D8156F3
:109120008A3150F589EAB82EBA0C8B2D90E08C1755
:109130009D0714F56F3FE1F0C216D306E406F5066D
:10914000B0F0CA01B901A40193010E9452459B01EC
:10915000AC012B0D311D411D511D2130F0E03F07A9
:10916000F0E04F07F0E85F0710F461E001C06FEF37
:10917000F801A1908F01C5CF2114310481F066233D
:1091800031F001501040F1010083118308C051FEFD
:109190001AC002501040F1010083118314C067FF10
:1091A00012C050FC05C02FEF3FEF4FEF5FE704C048
:1091B00020E030E040E050E882E290E080934830E8
:1091C0009093493016C050FE08C050954095309598
:1091D00021953F4F4F4F5F4F0CC057FF0AC082E2AF
:1091E00090E080934830909349302FEF3FEF4FEF5E
:1091F0005FE7B901CA01DF91CF911F910F91FF90F5
:10920000EF90DF90CF90BF90AF909F908F907F9026
:109210006F905F903F902F900895FC0188279927C9
:10922000E89421912032E9F3293010F02E30C8F370
:109230002B3241F02D3239F4689404C00E94C949A0
:10924000820F911D219120532A30C0F31EF4909576
:1092500081959F4F0895803209F09111F4C5805295
:109260008F55E0F708959111EEC5803219F08950BD
:109270008550D0F708959111089581548A5108F4CA
:10928000805E855A0895FB01DC0102C005900D92B5
:1092900041505040D8F70895FC0105900020E9F7AF
:1092A000809590958E0F9F1F089540E050E30E9497
:1092B000A2490895FB01DC0102C001900D924150CA
:1092C0005040D8F70895DC0101C06D9341505040E3
:1092D000E0F70895FB01DC010D900020E9F71197FC
:1092E00001900D920020E1F70895FB01DC018D91C2
:1092F000019080190110D9F3990B0895FB01DC014D
:1093000001900D920020E1F70895FB01DC0141502E
:10931000504030F08D910190801919F40020B9F778
:10932000881B990B0895FB01DC014150504048F027
:1093300001900D920020C9F701C01D92415050408C
:10934000E0F70895FA01A191B081009719F4109700
:10935000E1F0CD01DC01CD010D90002011F4C00140
:1093600013C0FB012191222319F02015D9F7F3CF67
:10937000FB012191201519F41E92119606C022239B
:10938000C1F70D900020A1F7D001FA01A193B0839D
:1093900008957AE0979F902D879F802D910D11243D
:1093A00008950F931F93DF93CF93CDB7DEB72E971A
:1093B000CDBFDEBF0E891F89888D998D97FF02C0B2
:1093C00080E090E801978D839E8309831A8386E06D
:1093D0008C839E01245E3F4FCE0101966A8D7B8D6A
:1093E000A9010E94574A4D815E8157FD0AC02F8115
:1093F0003885421753070CF49A01020F131FF80126
:1094000010822E96CDBFDEBFCF91DF911F910F91BD
:109410000895DF93CF93CDB7DEB72E97CDBFDEBFD4
:1094200085E08C838C899D8989839A839E01285E3F
:109430003F4FCE0101966E897F89A9010E94004E9F
:109440002E96CDBFDEBFCF91DF9108950F931F936E
:10945000DF93CF93CDB7DEB72E97CDBFDEBF8C01A4
:1094600077FF02C060E070E8615070406D837E83DA
:1094700009831A8386E08C83CE010196BA01A90183
:109480000E94574A2D813E8137FD09C0EF81F88542
:109490002E173F070CF4F901E00FF11F10822E96F2
:1094A000CDBFDEBFCF91DF911F910F9108952F9215
:1094B0003F924F925F926F927F928F929F92AF9264
:1094C000BF92CF92DF92EF92FF920F931F93DF93A1
:1094D000CF93CDB7DEB72B97CDBFDEBF3C012B01BD
:1094E0005A01FC0116821782838181FD03C06FEF50
:1094F0007FEFC6C19AE0892E1E010894211C311C01
:10950000F3012381F20123FD859123FF81912F0136
:10951000882309F4B2C1853239F423FD859123FFF4
:1095200081912F01853229F490E0B3010E94894F87
:10953000E7CF982FFF24EE249924FFE1FF15D0F008
:109540009B3269F09C3228F4903259F0933291F4B6
:109550000EC09D3249F0903369F441E024C052E0DE
:10956000F52A84E0F82A28C098E0F92A25C0E0E12D
:10957000FE2A22C0F7FC29C0892F80538A3070F45C
:10958000F6FE05C0989C902C1124980E15C0E89CFE
:10959000E02C1124E80EF0E2FF2A0EC09E3229F4DE
:1095A000F6FC6BC140E4F42A07C09C3619F450E87D
:1095B000F52A02C0983649F4F20123FD959123FF64
:1095C00091912F01992309F0B8CF892F85548330C9
:1095D00018F08052833038F444E050E0A40EB51EF9
:1095E0005FE359830FC0933631F0933779F09335A9
:1095F00009F056C020C0F5018081898342E050E027
:10960000A40EB51E610101E010E012C0F501C0809A
:10961000D180F6FC03C06FEF7FEF02C0692D70E0D0
:1096200042E050E0A40EB51EC6010E943C4F8C01E2
:109630005FE7F52214C0F501C080D180F6FC03C0BD
:109640006FEF7FEF02C0692D70E042E050E0A40EA2
:10965000B51EC6010E94314F8C0150E8F52AF3FE79
:1096600007C01AC080E290E0B3010E94894FEA94DB
:109670008E2D90E008171907A8F30EC0F601F7FC2D
:109680008591F7FE81916F0190E0B3010E94894FAF
:10969000E110EA94015010400115110579F7EAC074
:1096A000943611F0993669F5F7FE08C0F50120816E
:1096B00031814281538184E090E00AC0F5018081CC
:1096C00091819C01442737FD4095542F82E090E022
:1096D000A80EB91E9FE6F92257FF09C05095409584
:1096E000309521953F4F4F4F5F4FE0E8FE2ACA016A
:1096F000B901A1012AE030E00E94CF4FD82ED21844
:1097000040C0953729F41F2D1F7E2AE030E01DC090
:109710001F2D197F9F3661F0903720F4983509F09E
:10972000ACC00FC0903739F0983709F0A6C004C01C
:1097300028E030E00AC0106114FD146020E130E040
:1097400004C014FD166020E132E017FF08C0F501E7
:10975000608171818281938144E050E008C0F5010D
:1097600080819181BC0180E090E042E050E0A40E55
:10977000B51EA1010E94CF4FD82ED2188FE7F82E28
:10978000F122F6FE0BC05EEFF522D91438F4F4FE98
:1097900007C0F2FC05C08FEEF82202C01D2D01C0EB
:1097A000192DF4FE0DC0FE01ED0DF11D80818033F9
:1097B00019F499EEF92208C01F5FF2FE05C003C03C
:1097C0008F2D867809F01F5F0F2DF3FC14C0F0FE7B
:1097D0000FC01E1510F09D2C0BC09D2C9E0C911AD5
:1097E0001E2D06C080E290E0B3010E94894F1F5FEA
:1097F0001E15C0F304C01E1510F4E11A01C0EE24BA
:1098000004FF0FC080E390E0B3010E94894F02FF84
:109810001DC001FD03C088E790E00EC088E590E020
:109820000BC0802F867891F001FF02C08BE201C04F
:1098300080E2F7FC8DE290E0B3010E94894F06C000
:1098400080E390E0B3010E94894F9A94D914C0F349
:10985000DA94F101ED0DF11D808190E0B3010E94D9
:10986000894FDD20A9F706C080E290E0B3010E9495
:10987000894FEA94EE20C1F743CEF30166817781E8
:10988000CB012B96CDBFDEBFCF91DF911F910F9102
:10989000FF90EF90DF90CF90BF90AF909F908F9010
:1098A0007F906F905F904F903F902F900895FC01B4
:1098B00020FD08C023FD05C022FF02C07383628320
:1098C000518340830895EF92FF920F931F9344FFBB
:1098D00002C033E011C046FF02C034E00DC0DB011E
:1098E000FC01AA0FBB1FEE1FFF1F1094D1F76A0FD8
:1098F0007B1F8E1F9F1F31E0660F771F881F991FE8
:109900003150D1F77B018C01E20EF11C011D111DBC
:10991000A8019701B701CA011F910F91FF90EF9025
:1099200008950F931F93CF93DF938C01C8010E947A
:10993000474FEC0197FD08C00E943349892BB1F7CE
:10994000CE01B8010E94B54FCE01DF91CF911F919A
:109950000F910895AF92BF92CF92DF92EF92FF9254
:109960000F931F93CF93DF93EC01C62E5A01122F52
:109970000E94474FAC018B3219F08D3251F41068C0
:10998000CA9409F46DC0CE010E94474FAC0197FD07
:1099900067C06DEFD62ED1228D2D807301F5403337
:1099A000F1F4CA9409F447C0CE010E94474FAC01BC
:1099B00097FD41C082E0D82A483711F0483559F464
:1099C00080E4D82ACA94B9F1CE010E94474FAC0175
:1099D00099232CF430C0D6FC02C080E1D82AEE24B2
:1099E000FF248701242F2053283088F0D4FC09C09D
:1099F0002A3068F0D6FE05C02F7D822F8151863037
:109A000028F0CA01BE010E94B54F12C02750C801FC
:109A1000B7014D2D0E94634C7B018C0182E0D82A56
:109A2000CA9461F0CE010E94474FAC0197FFDACF94
:109A3000D1FC04C015C0EE24FF248701D7FE08C066
:109A400010950095F094E094E11CF11C011D111D8E
:109A5000C501B801A7012D2D0E94574C81E001C01E
:109A600080E0DF91CF911F910F91FF90EF90DF90F9
:109A7000CF90BF90AF9008956F927F928F929F92F8
:109A8000AF92BF92CF92DF92EF92FF920F931F930C
:109A9000DF93CF93CDB7DEB7A097CDBFDEBF6C010C
:109AA000A62E8A017901FE01319680E2DF011D9226
:109AB0008A95E9F770E030E060E040E050E04F0167
:109AC000A1E0B0E0F6018381F70183FD259183FFDA
:109AD00021917F01222309F47EC02E3519F441150E
:109AE000510569F1872F90E08417950744F42D35CF
:109AF00051F12D3221F4332329F431E021C03323F5
:109B000009F4622F322F832F869586958695F4016E
:109B1000E80FF11D832F87703D0102C0660C771C92
:109B20008A95E2F7208126292083361711F430E048
:109B300007C0361710F43F5FE6CF3150E4CF71E035
:109B40004F5F5F4FBFCF332319F08E8180628E83CA
:109B5000772359F0FE0131969E012F5D3F4F8081A2
:109B600080958193E217F307D1F7BB24B3944E019C
:109B70000894811C911CC6010E94474FAC0197FDBF
:109B800022C0869586958695F401E80FF11D8081A7
:109B900090E09A012770307002C0959587952A95BC
:109BA000E2F780FD05C0CA01B6010E94B54F0BC0A7
:109BB0000115110519F0D8014D938D01AA94BB240C
:109BC000AA20C9F602C0BB2031F40115110529F005
:109BD000F801108202C0EE24FF24C701A096CDBF79
:109BE000DEBFCF91DF911F910F91FF90EF90DF903B
:109BF000CF90BF90AF909F908F907F906F9008957F
:109C00006F927F928F929F92AF92BF92CF92DF928C
:109C1000EF92FF920F931F93CF93DF935C016B0141
:109C20003A01FC01168217828824EAC0812F90E055
:109C30000E943349892B21F0C5010E94914CE0C05C
:109C4000153249F4F601F3FC6591F3FE61916F0161
:109C5000653269F415E2C5010E94474F97FDDCC0EB
:109C6000181709F4CDC0B5010E94B54FDAC06A32A9
:109C700019F0162F00E006C0F3FC1591F3FE1191C8
:109C80006F0101E099240FC00260692D70E080E04F
:109C900090E040E20E94634C962EF601F3FC159191
:109CA000F3FE11916F01212F20532A3068F301FD3B
:109CB00003C099249A9403C0992009F4B2C01836BD
:109CC00021F01C3699F4F6010BC0F601F3FC659106
:109CD000F3FE6191683619F06F01162F07C0086016
:109CE0000460F3FC1591F3FE11916F01112309F447
:109CF00098C085E09FE0612F70E00E94264F892B7D
:109D000009F48FC0802F00FF03C0EE24FF2407C09A
:109D1000F301E080F18022E030E0620E731E1E3617
:109D200051F4F5014681578160E070E0C701202FB2
:109D30000E94574C65C0133691F481FD02C09924EE
:109D40009394C5010E94474F97FD66C0E114F1044A
:109D500019F0F70181937F019A9499F74FC01B3551
:109D600059F4C501692DA70196010E943C4D6C0173
:109D7000009709F043C03DC0C5010E94914C97FD7A
:109D80004BC01F3659F1103728F4143629F1193613
:109D900039F527C0133719F0153711F51DC0C50166
:109DA0000E94474FEC0197FD11C00E943349892B57
:109DB00029F0CE01B5010E94B54F08C0E114F104AD
:109DC00019F0F701C1937F019A9449F7E114F10466
:109DD000A9F0F701108212C0006203C0006101C047
:109DE0000064C501692DA701202F0E94AA4C882379
:109DF00029F4F5018381807379F413C000FF839403
:109E0000F501F380F601F3FC1591F3FE11916F015A
:109E1000112309F00BCF05C0882019F42FEF3FEF75
:109E200002C0282D30E0C901DF91CF911F910F9121
:109E3000FF90EF90DF90CF90BF90AF909F908F906A
:109E40007F906F900895992788270895FC010590C9
:109E5000061621F00020D9F7C00108953197CF01EF
:109E60000895FC010590615070400110D8F780956D
:109E700090958E0F9F1F0895FC01615070400190D6
:109E80000110D8F7809590958E0F9F1F0895CF935E
:109E9000DF93EC014B8140FF1AC046FF0AC04F7BA5
:109EA0004B838E819F8101968E839F838A81282F89
:109EB0002BC042FF13C0E881F9818081282F33270E
:109EC00027FD30952115310529F440624B832FEF92
:109ED0003FEF1BC03196E883F98311C0EA85FB850B
:109EE000CE0119959C0197FF0AC09B812F5F3F4FC0
:109EF00011F080E201C080E1892B8B83E8CF8E8155
:109F00009F8101968E839F8330E0C901DF91CF91BD
:109F100008950F931F93CF93DF938C01EB018B81F7
:109F200081FF1BC082FF0DC02E813F818C819D81EE
:109F30002817390764F4E881F9810193E883F983EC
:109F400006C0E885F985802F1995892B31F48E811B
:109F50009F8101968E839F8302C00FEF1FEFC80180
:109F6000DF91CF911F910F9108959C01FB01838197
:109F700080FF11C086FD0FC09FEF2F3F390759F0BA
:109F8000228380648F7D8383868197810197868376
:109F9000978330E002C02FEF3FEFC9010895FA0127
:109FA000AA27283051F1203181F1E8946F936E7F18
:109FB0006E5F7F4F8F4F9F4FAF4FB1E03ED0B4E009
:109FC0003CD0670F781F891F9A1FA11D680F791F4A
:109FD0008A1F911DA11D6A0F711D811D911DA11D5B
:109FE00020D009F468943F912AE0269F112430196B
:109FF000305D3193DEF6CF010895462F4770405D06
:10A000004193B3E00FD0C9F7F6CF462F4F70405DB4
:10A010004A3318F0495D31FD4052419302D0A9F70F
:10A02000EACFB4E0A6959795879577956795BA9509
:10A03000C9F700976105710508959B01AC010A2ECF
:10A0400006945795479537952795BA95C9F7620FA6
:0EA05000731F841F951FA01D0895F894FFCF65
:10A05E00200000252D3230732025730A0D002400B8
:10A06E00257320002573202D2068657864756D702A
:10A07E00286C656E3D2564293A0A0D00253032782C
:10A08E002000202020003A200020202025730A0DD9
:10A09E0000082008000A0D00636F6D6D616E64206C
:10A0AE006E6F7420666F756E643A25730A0D002507
:10A0BE00630068656C70007072696E7420746869F4
:10A0CE007320696E666F726D6174696F6E002573B1
:10A0DE00202D2068657864756D70286C656E3D2541
:10A0EE0064293A0A0D002530327820002020200005
:10A0FE003A200020202025730A0D007375636365D6
:10A10E00737300696E76616C696420706172616D43
:10A11E00657465727300756E6B6E6F776E20666117
:10A12E00696C757265006F7574206F66206D656D54
:10A13E006F72792F62756666657273006E6F74202A
:10A14E00636F6E6E656374656400696E76616C69CB
:10A15E00642073746174650070617273696E672038
:10A16E006572726F720070617468206E6F74206613
:10A17E006F756E6400696E636F6D70617469626C89
:10A18E00652074797065006E6F207065726D6973ED
:10A19E0073696F6E006F7065726174696F6E206E99
:10A1AE006F7420737570706F72746564006F757460
:10A1BE00206F662072616E6765006261642073694C
:10A1CE007A65007265747279206C617465720062D2
:10A1DE007573790064697361626C65640070726F87
:10A1EE00746F636F6C206572726F720074696D6547
:10A1FE006F75740069676E6F7265640063616E637C
:10A20E00656C65642062792072656D6F746500738C
:10A21E00796E63206572726F720061626F7274651F
:10A22E006400616C726561647920696E2075736576
:10A23E00002D2D2D20415353455254494F4E20464B
:10A24E0041494C4544202D2D2D0A0D002D412D2028
:10A25E0025733A25642025733A2025730A0D002EA6
:10A26E002E2F2E2E2F2E2E2F2E2E2F746F6F6C6BB9
:10A27E0069742F6F776C2F636F72652F6F776C5FBA
:10A28E006572722E63003000756E6B6E6F776E00A6
:10A29E002D2D2D20415353455254494F4E204641AA
:10A2AE00494C4544202D2D2D0A0D002D412D2025E4
:10A2BE00733A25642025733A2025730A0D002E2E3D
:10A2CE002F2E2E2F2E2E2F2E2E2F746F6F6C6B691E
:10A2DE00742F6F776C2F636F72652F6F776C5F744F
:10A2EE00696D65722E63002128746D6F2D3E666C4C
:10A2FE00616773202620544D4F5F44454C455445AD
:10A30E0044290045004E004F004D0053002D2D2DC9
:10A31E0020415353455254494F4E204641494C45D6
:10A32E0044202D2D2D0A0D002D412D2025733A256B
:10A33E00642025733A2025730A0D002E2E2F2E2E03
:10A34E002F2E2E2F2E2E2F746F6F6C6B69742F6F16
:10A35E00776C2F706F7274732F617672382F6F77E0
:10A36E006C5F756172742E630030000076657273D7
:10A37E00696F6E3A25642E25642E25640A0D0063DE
:10A38E006F6E6E5F636220736F636B69643A2564F0
:10A39E0020636F6E6E65637465643A25640A0D0002
:10A3AE00657272006F6B002573202564202825735B
:10A3BE00290A0D0076657273696F6E3A25642E2533
:10A3CE00642E2564206275696C643A25730A0D004B
:10A3DE0075736167653A206765745F686F73746241
:10A3EE00796E616D65203C646E736E616D653E0ABB
:10A3FE000D006C6F6F6B75705F63623A20686F73E0
:10A40E0074206E6F7420666F756E640A0D006C6F2B
:10A41E006F6B75705F63622069703A25730A0D0069
:10A42E002573202564202825732920007065657208
:10A43E003A25730A0D0075736167653A2067657476
:10A44E005F7065657261646472203C736F636B69E3
:10A45E00643E0A0D0073656E64696E672025642084
:10A46E00627974657320746F2025733A25640A0D22
:10A47E000077726F74653A25642072656D61696E3E
:10A48E003A25640A0D0075736167653A2073656E2F
:10A49E0064746F203C736F636B69643E203C69701B
:10A4AE003E203C706F72743E203C64617461202EBD
:10A4BE002E2E3E0A0D0073656E64696E672025644C
:10A4CE002062797465730A0D0075736167653A20B1
:10A4DE0073656E64203C736F636B69643E203C64ED
:10A4EE00617461202E2E2E3E0A0D00757361676514
:10A4FE003A20636C6F7365203C736F636B69643EC7
:10A50E000A0D0075736167653A20636F6E6E656341
:10A51E0074203C736F636B69643E203C69703E200F
:10A52E003C706F72743E0A0D0075736167653A2058
:10A53E006C697374656E203C736F636B69643E2047
:10A54E005B6261636B6C6F675D0A0D006C6973749F
:10A55E00656E5F636220736F636B69643A25642C6A
:10A56E0020616363657074696E67202E2E2E200045
:10A57E0028636F6E6E656374696F6E206C6F737493
:10A58E00290000726563765F636220736F636B6987
:10A59E00643A2564206C656E3A25642025730A0D95
:10A5AE000052580075736167653A2062696E6420C7
:10A5BE003C736F636B69643E203C69703E203C7057
:10A5CE006F72743E0A0D0073747265616D0064677C
:10A5DE0072616D007261770075736167653A207301
:10A5EE006F636B6574203C73747265616D7C646718
:10A5FE0072616D7C7261773E205B70726F746F63F7
:10A60E006F6C5D0A0D0075736167653A2073657432
:10A61E005F6468637064203C307C313E0A0D002517
:10A62E00732025642028656E61626C65643A25642A
:10A63E00290A0D0075736167653A207365745F644E
:10A64E00686370203C307C313E0A0D002573202556
:10A65E006420280069703A257320006D61736B3A8F
:10A66E002573200067773A25732000646E733A25B0
:10A67E0073290A0D0075736167653A207365745FFF
:10A68E00697061646472203C69703E205B6D617319
:10A69E006B5D205B67775D205B646E735D0A0D00FA
:10A6AE004E2F410025732025642028257320253048
:10A6BE0032783A253032783A253032783A253032AF
:10A6CE00783A253032783A25303278290A0D00252D
:10A6DE00732025642028253032783A253032783A96
:10A6EE00253032783A253032783A253032783A258C
:10A6FE00303278290A0D0075736167653A207365EB
:10A70E00745F6368616E6E656C203C6368616E6E2B
:10A71E00656C3E0A0D0061700073746100757361A3
:10A72E0067653A207365745F6D6F6465203C737462
:10A73E00617C736F667461703E0A0D00757361679C
:10A74E00653A206C696E6B7570205B737369645D1E
:10A75E00205B6B65795D205B7765705D0A0D00751A
:10A76E00736167653A207365745F626175647261C7
:10A77E007465203C62617564726174653E205B7223
:10A78E0074736374735D0A0D006572722025642004
:10A79E00286661696C656420746F20636F6E6669EC
:10A7AE006775726520686F73742075617274290AFB
:10A7BE000D00726573657400776C705F72657365FA
:10A7CE00742829007365745F6261756472617465C3
:10A7DE0000776C705F7365745F626175647261742B
:10A7EE00652829006C696E6B757000776C705F6CF4
:10A7FE00696E6B757028737369642C206B65792C88
:10A80E002077657029006C696E6B646F776E0077C8
:10A81E006C705F6C696E6B646F776E282900736560
:10A82E00745F6D6F646500776C705F7365745F6DD8
:10A83E006F64652829006765745F6D6F64650077C6
:10A84E006C705F6765745F6D6F6465282900736552
:10A85E00745F6368616E6E656C00776C705F7365B4
:10A86E00745F6368616E6E656C2829006765745F3E
:10A87E0068776164647200776C705F6765745F6897
:10A88E0077616464722829006765745F6E657477FA
:10A89E006F726B00776C705F6765745F6E6574774F
:10A8AE006F726B2829007365745F697061646472DE
:10A8BE0000776C705F7365745F6970616464722891
:10A8CE0069702C206D61736B2C2067772C20646E61
:10A8DE007329006765745F69706164647200776CD8
:10A8EE00705F6765745F69706164647228290073B4
:10A8FE0065745F6468637000776C705F7365745F16
:10A90E006468637028656E61626C652900676574A2
:10A91E005F6468637000776C705F6765745F64680E
:10A92E0063702829007365745F64686370640077D0
:10A93E006C705F7365745F6468637064282900735C
:10A94E006F636B657400776C705F736F636B6574A8
:10A95E0028747970652C2070726F746F290062698B
:10A96E006E6400776C705F62696E6428736F636BE0
:10A97E002C2069702C20706F727429006C697374AE
:10A98E00656E00776C705F6C697374656E28736F9B
:10A99E00636B69642C206261636B6C6F6729006363
:10A9AE006F6E6E65637400776C705F636F6E6E654D
:10A9BE00637428736F636B69642C2069702C20702C
:10A9CE006F72742900636C6F736500776C705F63D0
:10A9DE006C6F736528736F636B6964290073656EA2
:10A9EE006400776C705F73656E6428736F636B6958
:10A9FE00642C2064617461290073656E64746F0049
:10AA0E00776C705F73656E64746F28736F636B69B8
:10AA1E00642C20646174612C2069702C20706F721C
:10AA2E007429006765745F70656572616464720095
:10AA3E00776C705F6765745F706565726164647270
:10AA4E0028736F636B696429006765745F686F7341
:10AA5E007462796E616D6500776C705F6765745FA7
:10AA6E00686F737462796E616D6528646E736E6162
:10AA7E006D6529006765745F66775F7665727369C9
:10AA8E006F6E00776C705F6765745F66775F766573
:10AA9E007273696F6E28636F64652C206275696CC2
:10AAAE006429006765745F76657273696F6E0070F6
:10AABE0072696E742076657273696F6E000A0D008E
:10AACE0074746370206572723A2564202825732988
:10AADE000A0D0074746370206F6B3A202564206237
:10AAEE00797465732070726F636573736564206922
:10AAFE006E20256C75206D732C20256C752E256CA3
:10AB0E0075204B422F730A0D0074746370206F6BA7
:10AB1E003A2025642062797465732070726F6365C4
:10AB2E007373656420696E2030206D730A0D002EDC
:10AB3E00002D2D2D20415353455254494F4E204642
:10AB4E0041494C4544202D2D2D0A0D002D412D201F
:10AB5E0025733A25642025733A2025730A0D002E9D
:10AB6E002E2F2E2E2F776C705F747463702E6300F1
:10AB7E00707269762D3E73656E6400706F73203D42
:10AB8E003D20707269762D3E6275666C656E002D85
:10AB9E0070002D6E002D6C002D74002D720025732B
:10ABAE0020256420282573290A0D00657272007411
:10ABBE0074637020636F6E6E6563742025733A251F
:10ABCE0064206E6275663A2564206275666C656EE9
:10ABDE003A256420736F636B69643A25640A0D002D
:10ABEE0074746370206C697374656E20706F727408
:10ABFE003A2564206275666C656E3A2564206C7326
:10AC0E006F636B69643A25640A0D0075736167653D
:10AC1E003A2074746370205B2D7472706E6C5D0AD2
:10AC2E000D00747463700074746370207468726FB6
:10AC3E007567687075742074657374006661696CED
:10AC4E00656420746F20676574206E74702074695B
:10AC5E006D653A2573282564290A0D006E747020DF
:10AC6E0074696D653A20253034642D253032642D9B
:10AC7E002530326420253032643A253032643A254C
:10AC8E003032640A0D00657272006F6B00257320FE
:10AC9E00256420282573290A0D0075736167653AAE
:10ACAE00206E7470203C6E74702D736572766572B2
:10ACBE003E0A0D006E7470006765742073657276BF
:10ACCE0065722074696D652066726F6D206E74708A
:10ACDE00002D2D2D2025732070696E6720737461F1
:10ACEE0074697374696373202D2D2D0A0D0025640C
:10ACFE00207061636B657473207472616E736D691D
:10AD0E00747465642C2025642072656365697665AC
:10AD1E00640A0D0025642062797465732066726F73
:10AD2E006D2025733A2069636D705F7365713D25E3
:10AD3E00640A0D0025642062797465732066726F53
:10AD4E006D2025733A2069636D705F7365713D25C3
:10AD5E00642044657374696E6174696F6E20486F08
:10AD6E00737420556E726561636861626C650A0D5D
:10AD7E000025642062797465732066726F6D2025DC
:10AD8E00733A2069636D705F7365713D256420545D
:10AD9E007970653A25640A0D002D63002D730065E8
:10ADAE007272006F6B00257320256420282573298D
:10ADBE000A0D0075736167653A2070696E67205BD6
:10ADCE002D63203C636F756E743E5D205B2D73208A
:10ADDE003C73697A653E5D203C69703E0A0D0070D9
:10ADEE00696E67004E2F4100253032783A25303299
:10ADFE00783A253032783A253032783A2530327822
:10AE0E003A253032780025642043002F002F3F0072
:10AE1E002F696E6465782E68746D6C3F00746F6771
:10AE2E00676C653D4C45442564002F696E646578FA
:10AE3E002E68746D6C002F6C6F676F2E67696600DD
:10AE4E000D0A0047455420006864776972656C6589
:10AE5E007373006864776972656C6573733132332E
:10AE6E00006C696E6B5F6362206C696E6B3A256471
:10AE7E000A0D00616464725F63622069703A6E6FDE
:10AE8E006E650A0D0068747470642073746F707050
:10AE9E0065640A0D00616464725F63622069703AD2
:10AEAE0025730A0D00687474706420737461727473
:10AEBE0065640A0D0020004A3000006220241B67E2
:10AECE00200000000062279F3268270000000074F7
:10AEDE0027C731812700000000942714319B2700DB
:10AEEE00000000B627D830BF2700000000CE277024
:10AEFE0030D72700000000E6272F30EF2700000094
:10AF0E0000FE27C32F0A28000000001C28772F27D9
:10AF1E0028000000003828D12E44280000000056DA
:10AF2E0028142E6128000000008328602D8E280032
:10AF3E000000009F28F32CA82800000000BD28B6B2
:10AF4E002CC62800000000D528492CDF2800000060
:10AF5E0000EF289F2BF628000000000E29082B1367
:10AF6E0029000000002C29B3293329000000004FCE
:10AF7E00291C295729000000007529AF287B2900BC
:10AF8E000000008D29C327922900000000A9299AEC
:10AF9E0026B02900000000D3290B26E0290000006E
:10AFAE0000F9294C25082A00000000242AAC24337D
:10AFBE002A00000000532A2C245F2A00000000D231
:10AFCE002B5836D72B00000000642C463B682C0013
:10AFDE000000008F2D7B3D8F2D0000000000000033
:10AFEE0000FFFFFFFF6F776C5F6572726F72006F0D
:10AFFE00776C746D725F64656C746D6F006F776CD7
:10B00E00756172745F70617269747900636F6E6ED0
:10B01E005F63620073656E646275660000001F00F8
:10B02E003B005A0078009700B500D400F3001101E0
:10B03E0030014E016D0100001F003C005B007900E5
:10B04E009800B600D500F400120131014F016E01D7
:00000001FF
